:020000040000FA
:1000000075EF3BF012001200BEEF01F0120001008C
:100010006C770000E3070000650100000F0E9316E7
:1000200081160ED9939493968194819609D90F0ED7
:100030008114816E300E8110816E2BD801D90F0E84
:100040008116300E811225D8FBD80F0E8116300E86
:10005000811246D91ED819D90F0E811641D9818A2D
:100060003FD917D8280EE66E19D8E552080EE66E6D
:1000700015D8E552010EE66E11D8E552060EE66E71
:100080000DD8E5520C0EE66E09D8E55229D900D0FC
:100090001200818625D981966AEF01F0D9CFE6FF5B
:1000A000E1CFD9FF1DD9819481960F0E8116FE0EE6
:1000B000DB50F00B811214D9ECDF0F0E8116FE0E0F
:1000C000DB38F00BF00B81120BD9E3DF00D0E552E7
:1000D000E7CFD9FF1200D9CFE6FFE1CFD9FF00D992
:1000E000818481960F0E8116FE0EDB50F00B81127B
:1000F0008186F6D881960F0E8116FE0EDB38F00B46
:10010000F00B81128186ECD8819600D0E552E7CFC2
:10011000D9FF1200D9CFE6FFE1CFD9FFFD0EDBCF2B
:10012000F6FFFE0EDBCFF7FF0800F55011E0FD0EE5
:10013000DBCFF6FFFE0EDBCFF7FF0800F550E66ED3
:10014000CADFE552FD0EDB2AFE0E01E3DB2AE6D70D
:1001500000D0E552E7CFD9FF1200D9CFE6FFE1CFBB
:10016000D9FFFD0EDBCFE9FFFE0EDBCFEAFFEF503C
:1001700010E0FD0EDBCFE9FFFE0EDBCFEAFFEF5014
:10018000E66EA9DFE552FD0EDB2AFE0E01E3DB2A57
:10019000E8D700D0E552E7CFD9FF1200D9CFE6FF6C
:1001A000E1CFD9FFE652FE0EDB0404E1FD0EDB5089
:1001B000800FDF6EFE0EDB50020804E1FD0EDB5007
:1001C000C00FDF6EDFCFE6FF69DFE552E552E55293
:1001D000E7CFD9FF1200D9CFE6FFE1CFD9FF020E5A
:1001E000E126E66AFE0EDBCFE6FFD8DFE552E552F8
:1001F000DE6ADD6ADECF14F0DDCF15F0D890155041
:1002000004E6100E145C000E155809E2200EE66E8E
:1002100062DFE552DF2A010E01E3DB2AEBD7E66A53
:10022000FE0EDBCFE6FFBADFE552E552020EE15CDF
:1002300002E2E16AE552E16EE552E7CFD9FF120032
:10024000D9CFE6FFE1CFD9FF020EE126DE6ADD6AF3
:10025000DECF14F0DDCF15F0D890155004E6100E67
:10026000145C270E155806E20000DF2A010E01E398
:10027000DB2AEED700D0020EE15C02E2E16AE55231
:10028000E16EE552E7CFD9FF1200D9CFE6FFE1CF0B
:10029000D9FF020EE126DE6ADD6ADECF14F0DDCF83
:1002A00015F0D890155004E6C40E145C090E1558CC
:1002B00006E20000DF2A010E01E3DB2AEED700D0C0
:1002C000020EE15C02E2E16AE552E16EE552E7CF3F
:1002D000D9FF120000000000000000000000120022
:1002E000D9CFE6FFE1CFD9FF020EE126DE6ADD6A53
:1002F000DECF14F0DDCF15F0D890155004E6E80EEF
:10030000145C030E155806E20000DF2A010E01E31B
:10031000DB2AEED700D0020EE15C02E2E16AE55290
:10032000E16EE552E7CFD9FF1200D9CFE6FFE1CF6A
:10033000D9FF81940F0E8116FE0EDB504009F00BA1
:100340008112C8DFA6DE0F0E8116FE0EDB38F00B21
:10035000F00B8112BFDF9DDE00D0E552E7CFD9FF61
:10036000120000000000000000000000000000007B
:10037000000000000000000000001200DACFE4FFDF
:10038000E2CFDAFFE9CFE4FFEACFE4FFF6CFE4FF04
:10039000F7CFE4FFF5CFE4FFF3CFE4FFF4CFE4FFC2
:1003A000FACFE4FF00EE00F0140EE80403E3EECF12
:1003B000E4FFFBD700EE14F0140EE80403E3EECFE5
:1003C000E4FFFBD7E6529D50200B30E09E50200BFF
:1003D0002DE0CFEC3AF00701116FABA407D0AB9E34
:1003E000D0810F2B000E1023AB8E01D0D091ABA289
:1003F00007D0AB98D083AB880D2B000E0E2301D015
:10040000D093ACA2FED7070104C7E9FF05C7EAFFF6
:10041000042B000E052311C7EFFFA00E045D000E94
:10042000055904E3600E046F000E056F9D50010B2B
:100430001CE09E50010B19E00701D12B000ED223C6
:10044000140ED15D000ED25907E3D16BD26BD0856B
:10045000D52B000ED6238978DB0EE66E0B0EE66EEA
:10046000EEEC3AF0E552E5529E90F250100B60E04F
:10047000F250020B5DE0070111510CE11B0E116FF0
:100480009D9A9E9A600E046F000E056F04C702F7D6
:1004900005C703F7F292F298A09CA19CA09AA19A9A
:1004A000010ED76FD86BCF8F9D9A070E961901E179
:1004B000975133E0060E961901E1975125E0010EA0
:1004C000961901E1975115E0020E961901E1975135
:1004D00010E0030E961901E197510BE0040E9619F6
:1004E00001E1975106E0050E961901E1975101E0EF
:1004F00016D099EC12F05CEC11F096C798F797C7FC
:1005000099F778EC1CF00BD0A3EC10F096C798F795
:1005100097C799F778EC1CF002D09AD900D0070160
:10052000D76BD86BF292F2889D8AA08CA08A116B4F
:10053000A050400B10E0A150400B0DE077AE04D06E
:10054000010E07019A6F9B6BA09CA19C07011B0EDB
:10055000116FB9EC1CF0A050200B10E0A150200B43
:100560000DE077AC04D0010E07019C6F9D6BA09A43
:10057000A19A07011B0E116FB9EC1CF0E55200EEB9
:1005800027F0140EE80403E3E5CFEDFFFBD700EE00
:1005900013F0140EE80403E3E5CFEDFFFBD7E5CF3E
:1005A000FAFFE5CFF4FFE5CFF3FFE5CFF5FFE5CFA9
:1005B000F7FFE5CFF6FFE5CFEAFFE5CFE9FFE5CFAF
:1005C000DAFF1100D9CFE6FFE1CFD9FFE6528B9ACF
:1005D0008B968B988B988B968B9A010EE66E91EC8E
:1005E0003BF0E5528B8A8B9A8B86010EE66E91EC7E
:1005F0003BF0E5528B96010EE66E91EC3BF0E55236
:100600008B8A010EE66E91EC3BF0E5528B9A010E5F
:10061000E66E91EC3BF0E552030EDF6E8B988B8615
:10062000010EE66E91EC3BF0E5528B96010EE66E04
:1006300091EC3BF0E552DF06DF500008EFE3010EDE
:10064000E66E91EC3BF0E5528B9A010EE66E91EC72
:100650003BF0E5528B8A010EE66E91EC3BF0E552E1
:100660008B9A010EE66E91EC3BF0E552E552E552B5
:10067000E7CFD9FF1200D9CFE6FFE1CFD9FFFB0EBC
:10068000DBCF14F0FC0EDBCF15F0FD0EDBCF16F048
:10069000FE0EDBCF17F080C70CF081C70DF082C7CC
:1006A0000EF083C70FF014C007F015C008F016C095
:1006B00009F017C00AF0E4EC2DF0CDEC2EF006C0E6
:1006C000CBF707C0CCF708C0CDF709C0CEF7CBC732
:1006D000E6FF32D8E552CCC7E6FF2ED8E552CDC7AB
:1006E000E6FF2AD8E552CEC7E6FF26D8E552C6C7B0
:1006F000E6FF22D8E552010EE66E91EC3BF0E552A2
:100700008B8A050EE66E91EC3BF0E5528B9A050E56
:10071000E66E91EC3BF0E5528B8A050EE66E91ECAD
:100720003BF0E5528B9A050EE66E91EC3BF0E552FC
:10073000E552E7CFD9FF1200D9CFE6FFE1CFD9FFCD
:10074000E652080EDF6E8B98FE0EDBB08B88DB4026
:100750007F0BE76EFE0EE7CFDBFF8B86010EE66EAA
:1007600091EC3BF0E5528B96DF06DF500008EBE39F
:10077000E552E552E7CFD9FF12000701CF8F010EF6
:10078000E66E29DDE552070EE66EE66ACBDBE55242
:10079000E55284C774F785C775F786C776F787C7AC
:1007A00077F7020EE66E17DDE552010EE66E29C9F7
:1007B000E6FF2AC9E6FF74C7E6FF75C7E6FF76C7FE
:1007C000E6FF77C7E6FF27EC09F0146E070EE15E3F
:1007D0001450030EE66E020EE66EE0DCE552E552C2
:1007E00029C9E6FF2AC9E6FFC5EC39F0E552E55212
:1007F000F3CF14F7F4CF15F707010A0ED88014577A
:10080000000E1557070114C714F015C715F014078B
:10081000000E155BD8801454000E155405E2200E0E
:10082000E66E59DCE552EED729C9E6FF2AC9E6FF94
:1008300094DCE552E552200EE66E4DDCE552480EA2
:10084000E66E49DCE5527A0EE66E45DCE5521200B2
:100850000701CF8F010EE66EBEDCE5520B0EE66E91
:10086000E66A60DBE552E55284C7E6FF85C7E6FF2E
:1008700086C7E6FF87C7E6FF0BEC38F0E552E55286
:10088000E552E55206C014F007C015F008C016F096
:1008900009C017F014C007F015C008F016C009F021
:1008A00017C00AF0CDEC2EF006C0AEF707C0AFF7C8
:1008B00008C0B0F709C0B1F7E66A2D0EE66E310E3A
:1008C000E66E010EE66EE66EE66AE66AE66AAEC7B8
:1008D000E6FFAFC7E6FFB0C7E6FFB1C7E6FF7AECB9
:1008E00017F0146E0C0EE15E145006C0AEF707C090
:1008F000AFF708C0B0F709C0B1F70701CF8F010EFD
:10090000E66E69DCE5520B0EE66EE66A0BDBE5523D
:10091000E552020EE66E5FDCE552AEC706F0AFC7E9
:1009200007F0B0C708F0B1C709F0DFEC2CF007C042
:1009300084F708C085F709C086F70AC087F7090160
:10094000D90E296F080E2A6F010EE66E29C9E6FF3F
:100950002AC9E6FF84C7E6FF85C7E6FF86C7E6FF2C
:1009600087C7E6FF27EC09F0146E070EE15E14500E
:1009700029C9E6FF2AC9E6FFADEC00F0E552E552D1
:10098000200EE66E6BEC00F0E552480EE66E6BEC66
:1009900000F0E5527A0EE66E6BEC00F0E55284C78B
:1009A000E6FF85C7E6FF86C7E6FF87C7E6FF63DE8B
:1009B000E552E552E552E5520701CF9F080EE66E7B
:1009C000E66AB0DAE552E5520901D90E296F080E40
:1009D0002A6F010EE66E29C9E6FF2AC9E6FF84C721
:1009E000E6FF85C7E6FF86C7E6FF87C7E6FF27EC79
:1009F00009F0146E070EE15E145029C9E6FF2AC9FA
:100A0000E6FF5AD9E552E552F3CF16F7F4CF17F7C0
:100A10009AD90701CF8F980EE66E3A0EE66EE66A17
:100A2000E66ACEEC0DF0E552E552E552E55298C784
:100A300096F799C797F778EF1CF0D9CFE6FFE1CF8B
:100A4000D9FF040EE126D9CFE9FFDACFEAFFFB0E8A
:100A5000DBCFEEFFFC0EDBCFEEFFFD0EDBCFEEFFBC
:100A6000FE0EDBCFEEFFD90EE66E080EE66ED9CF96
:100A7000E9FFDACFEAFFEECFE6FFEECFE6FFEECFFB
:100A8000E6FFEFCFE6FFEAEC34F0146E060EE15E0F
:100A90001450D90EE66E080EE66E0ED9E552E552F8
:100AA000F3CF16F7F4CF17F7090EE66E3CD9E552EF
:100AB000D9CFE9FFDACFEAFFEECF14F0EECF15F091
:100AC000EECF16F0EFCF17F01450E66E76EC0DF087
:100AD000E552090EE66E27D9E552D9CFE9FFDACF04
:100AE000EAFFEECF14F0EECF15F0EECF16F0EFCF19
:100AF00017F0080ED8901732163215321432E80665
:100B0000F9E114C0DFFF010E15C0DBFF020E16C0B5
:100B1000DBFF030E17C0DBFFD9CFE9FFDACFEAFF17
:100B2000EECF14F0EECF15F0EECF16F0EFCF17F0BA
:100B30001450E66E76EC0DF0E552090EE66EF3D831
:100B4000E552000EDFCFE6FF76EC0DF0E552090E20
:100B5000E66EE9D8E552D9CFE9FFDACFEAFFEECF6A
:100B600014F0EECF15F0EECF16F0EFCF17F0080E21
:100B7000D8901732163215321432E806F9E114C053
:100B8000DFFF010E15C0DBFF020E16C0DBFF030EF8
:100B900017C0DBFFD9CFE9FFDACFEAFFEECF14F0C1
:100BA000EECF15F0EECF16F0EFCF17F01450E66E43
:100BB00076EC0DF0E552090EE66EB5D8E552D9CFC8
:100BC000E9FFDACFEAFFEECF14F0EECF15F0EECF6B
:100BD00016F0EFCF17F0080ED890173216321532F4
:100BE0001432E806F9E114C0DFFF010E15C0DBFF87
:100BF000020E16C0DBFF030E17C0DBFF000EDFCFB7
:100C0000E6FF76EC0DF0E552090EE66E8CD8E55263
:100C10009AD8040EE15C02E2E16AE552E16EE55227
:100C2000E7CFD9FF1200800EE66EE66A740EE66E1C
:100C30003AEC3AF0E552E552E5529F8AD08E9D9A01
:100C4000F29CF29E1200D9CFE6FFE1CFD9FF020E4F
:100C5000E126DE6ADD6AFD0EDBCFF6FFFE0EDBCF9E
:100C6000F7FF0800F55015E0FD0EDBCFF6FFFE0E96
:100C7000DBCFF7FF0800F550E66E55D8E552DF2AC6
:100C8000010E01E3DB2AFD0EDB2AFE0E01E3DB2A67
:100C9000E2D7DECF14F0DDCF15F014C0F3FF15C09E
:100CA000F4FF020EE15C03E200D0E16AE552E16E7E
:100CB000E552E7CFD9FF1200D9CFE6FFE1CFD9FF48
:100CC000020EE126DE6ADD6AFD0EDBCFE9FFFE0ED5
:100CD000DBCFEAFFEF5014E0FD0EDBCFE9FFFE0EA5
:100CE000DBCFEAFFEF50E66E1ED8E552DF2A010E99
:100CF00001E3DB2AFD0EDB2AFE0E01E3DB2AE4D74B
:100D0000DECF14F0DDCF15F014C0F3FF15C0F4FFF3
:100D1000020EE15C03E200D0E16AE552E16EE552C9
:100D2000E7CFD9FF1200D9CFE6FFE1CFD9FFACA2C0
:100D3000FED7FE0EDBCFE6FF26EC3BF0E552E55298
:100D4000E7CFD9FF12000D0EE66EEDDFE5520A0E79
:100D5000E66EE9DFE5521200D9CFE6FFE1CFD9FF19
:100D6000E65207010451021902E10551031901E19C
:100D7000F8D702C7E9FF03C7EAFF022B000E0323DF
:100D8000EFCFDFFFA00E025D000E035904E3600EFB
:100D9000026F000E036FDF5000D0E552E552E7CF3F
:100DA000D9FF1200D9CFE6FFE1CFD9FFFF0EE76EE2
:100DB000FD0EDBCF14F0FE0EDBCF15F0E75014165E
:100DC000156A1450A96EFD0EDBCF14F0FE0EDBCFBA
:100DD00015F015C014F0156A030E1414AA6EA69E21
:100DE000A69CA680E80EE66E030EE66EE66AE66A4C
:100DF000CEEC0DF0E552E552E552E552A85000D098
:100E0000E552E7CFD9FF1200D9CFE6FFE1CFD9FFF6
:100E1000020EE1260701CFAF11D0E76EFD0EDBCF4A
:100E200014F0FE0EDBCF15F0E7501426000E15224D
:100E3000FD0E14C0DBFFFE0E15C0DBFFFD0EDBCF89
:100E400014F0FE0EDBCF15F015C014F0156A030E7A
:100E50001414AA6EFF0EE76EFD0EDBCF14F0FE0E2B
:100E6000DBCF15F0E7501416156A1450A96EFC0E6E
:100E7000DB50A86EA69EA684A69CF2AE04D0F29E7D
:100E8000010EDE6EDD6A550EA76EAA0EA76EA68253
:100E9000A1A8FED7A198A694D9CFE9FFDACFEAFF9F
:100EA000010EEE1801E1ED5001E1F28E020EE15C5F
:100EB00002E2E16AE552E16EE552E7CFD9FF1200A6
:100EC000D9CFE6FFE1CFD9FFFB0EDBCFE9FFFC0E68
:100ED000DBCFEAFFEF5022E0FB0EDBCFE9FFDB2A9E
:100EE000FC0EDBCFEAFF01E3DB2AEF50E66ED950C0
:100EF000FD0FE96EFF0EDA20EA6EEECF14F0EDCFB3
:100F000015F0020EEE26000EEF2214C0E6FF15C00B
:100F1000E6FF7ADFE552E552E552D6D7E552E7CF54
:100F2000D9FF1200D9CFE6FFE1CFD9FF040EE126A9
:100F30000701CFAF17D0FD0EDBCF14F0FE0EDBCFD5
:100F400015F0040ED89014361536E804FBE1000EB7
:100F50001426020E1522FD0E14C0DBFFFE0E15C076
:100F6000DBFF12D0FD0EDBCF14F0FE0EDBCF15F051
:100F7000050ED89014361536E804FBE1FD0E14C0BA
:100F8000DBFFFE0E15C0DBFF020EDB6A030EDB6A21
:100F9000D950FD0FE96EFF0EDA20EA6EFF0ED88001
:100FA000EE54030EED5401E242D0FD0EDBCFE6FF1E
:100FB000FE0EDBCFE6FFF6DEE552E552DE6EDD6AC1
:100FC000D9CFE9FFDACFEAFFEE50ED1001E12FD0E3
:100FD0000701CF51800B0EE0020EDBCF14F0030EA1
:100FE000DBCF15F0153404E214500F08000E155431
:100FF00001E21DD0CFBF05D0DFCFE6FF94DEE55282
:1010000005D0DFCFE6FF6BEC00F0E552FD0EDB2AEA
:10101000FE0E01E3DB2A020EDB2A030E01E3DB2ACC
:10102000D9CFE9FFDACFEAFFEE50ED10B1E1E80EDB
:10103000E66E030EE66EE66AE66ACEEC0DF0E55269
:10104000E552E552E552040EE15C02E2E16AE55246
:10105000E16EE552E7CFD9FF1200D9CFE6FFE1CF2D
:10106000D9FF0A0EE12607012B0E006F090E016F52
:10107000FC0EDB50010801E2E0D0FC0EDB5028E161
:10108000FD0EDBCF14F0FE0EDBCF15F0060E14C004
:10109000DBFF070E15C0DBFF080EDB6A090EDB6AFB
:1010A00000C7E6FF01C7E6FFD950060FE96EDACFA9
:1010B000EAFFEECFE6FFEECFE6FFEECFE6FFEFCFA3
:1010C000E6FFEAEC34F0146E060EE15E145010D028
:1010D00000C7E6FF01C7E6FFFD0EDBCFE6FFFE0E11
:1010E000DBCFE6FF50EC34F0E552E552E552E55235
:1010F0000701D0AD80D000C7E6FF01C7E6FFC5EC11
:1011000039F0E552E552020EF3CFDBFF030EF4CFC8
:10111000DBFFDE6ADD6ADECF14F0DDCF15F0020EF4
:10112000DBCF16F0030EDBCF17F01650145C175010
:1011300015582CE2020EDBCF16F0030EDBCF17F0B2
:10114000DE50165CE96EDD501758EA6EE906000EB7
:10115000EA5A2B0EE926090EEA22EF50E66EFC0E43
:10116000DB50040F146E156ADE50145CE96EDD501E
:101170001558EA6E2B0EE926090EEA22E552E750D1
:10118000EF6EDF2A010E01E3DB2AC5D7DE6ADD6AD6
:10119000DECF14F0DDCF15F0FC0EDB50050F186E1E
:1011A000196A020EDB50185C166E030EDB501958DC
:1011B000176E1650145C175015581DE20701D0A980
:1011C0000BD0DECFE9FFDDCFEAFF2B0EE926090EBB
:1011D000EA22300EEF6E0AD0DECFE9FFDDCFEAFF64
:1011E0002B0EE926090EEA22200EEF6EDF2A010EF1
:1011F00001E3DB2ACDD7FC0EDB50050FEA6A2B0F8B
:10120000E96E090EEA22EF6A0701CFAF09D000C7E5
:10121000E6FF01C7E6FFADEC00F0E552E5520DD068
:1012200000C7E6FF01C7E6FF47DDE552E552020EC3
:10123000F3CFDBFF030EF4CFDBFF0A0EE15C02E22B
:10124000E16AE552E16EE552E7CFD9FF1200D9CF4E
:10125000E6FFE1CFD9FF0E0EE126F90EDBCFDEFF70
:10126000DBCFDDFFF80EDB50000802E3070E08D0ED
:10127000F80EDB50160802E2170E02D0F80EDB283B
:10128000E66ED950080FE96EDACFEAFFE552E75073
:10129000EE6EED6A020EDB6A030EDB6AFB0EDBCF3D
:1012A00014F0FC0EDBCF15F0FD0EDBCF16F0FE0EBA
:1012B000DBCF17F00C6A0D6A0E6A0F6A14C007F0D4
:1012C00015C008F016C009F017C00AF00DEC2FF099
:1012D000010A33E1F90EDBCFE9FFDB2AFA0EDBCF9F
:1012E000EAFF01E3DB2A2D0EEF6EFB0EDBCF14F0DD
:1012F000FC0EDBCF15F0FD0EDBCF16F0FE0EDBCFC4
:1013000017F00C6A0D6A800E0E6EBF0E0F6E14C0C1
:1013100007F015C008F016C009F017C00AF0E4EC99
:101320002DF0FB0E07C0DBFFFC0E08C0DBFFFD0E3F
:1013300009C0DBFFFE0E0AC0DBFFFB0EDBCF14F0A3
:10134000FC0EDBCF15F0FD0EDBCF16F0FE0EDBCF73
:1013500017F00C6A0D6A0E6A0F6A14C007F015C008
:1013600008F016C009F017C00AF004EC2FF0010ACB
:101370004AE1FB0EDBCF14F0FC0EDBCF15F0FD0EC7
:10138000DBCF16F0FE0EDBCF17F00C6A0D6A800E75
:101390000E6E3F0E0F6E14C007F015C008F016C099
:1013A00009F017C00AF00DEC2FF0010A2CE1146AC5
:1013B000156A200E166E410E176ED950FB0FE96E9E
:1013C000FF0EDA20EA6EEECF07F0EECF08F0EECF98
:1013D00009F0EFCF0AF014C00CF015C00DF016C0E4
:1013E0000EF017C00FF0E4EC2DF00AC0EDFF09C0BD
:1013F000EDFF08C0EDFF07C0EFFF020EDB06030E96
:1014000001E2DB06B6D7FB0EDBCF14F0FC0EDBCF20
:1014100015F0FD0EDBCF16F0FE0EDBCF17F00C6AD9
:101420000D6A200E0E6E410E0F6E14C007F015C02F
:1014300008F016C009F017C00AF00DEC2FF0010AF1
:101440002EE0FB0EDBCF14F0FC0EDBCF15F0FD0E13
:10145000DBCF16F0FE0EDBCF17F00C6A0D6A200E04
:101460000E6E410E0F6E14C007F015C008F016C0C6
:1014700009F017C00AF091EC2DF0FB0E07C0DBFF5E
:10148000FC0E08C0DBFFFD0E09C0DBFFFE0E0AC02C
:10149000DBFF020EDB2A030E01E3DB2AB4D7020EC8
:1014A000DBCF14F0030EDBCF15F0D950080FE96E37
:1014B000DACFEAFF1450EE261550ED22010EF36E3E
:1014C000040EF3CFDBFF050EDB6A040EDBCF08F062
:1014D000050EDBCF09F0CCEC2CF00A0E07C0DBFFC9
:1014E0000B0E08C0DBFF0C0E09C0DBFF0D0E0AC09F
:1014F000DBFF040EDBCF14F0050EDBCF15F0080E7A
:10150000DBCF16F0090EDBCF17F015501718E8AE39
:1015100002D0173404D01650145C175015582EE220
:101520000A0EDBCF14F00B0EDBCF15F00C0EDBCF69
:1015300016F00D0EDBCF17F00C6A0D6A200E0E6E42
:10154000410E0F6E14C007F015C008F016C009F068
:1015500017C00AF091EC2DF00A0E07C0DBFF0B0E4E
:1015600008C0DBFF0C0E09C0DBFF0D0E0AC0DBFF5D
:10157000040EDB2A050E01E3DB2ABBD70A0EDBCF04
:1015800018F00B0EDBCF19F00C0EDBCF1AF00D0E9E
:10159000DBCF1BF00C6A0D6A0E6A400E0F6E18C08E
:1015A00007F019C008F01AC009F01BC00AF091EC4E
:1015B0002DF007C014F008C015F009C016F00AC0DD
:1015C00017F0D950FB0FE96EFF0EDA20EA6EEECF6E
:1015D00007F0EECF08F0EECF09F0EFCF0AF014C01D
:1015E0000CF015C00DF016C00EF017C00FF0FBEC9C
:1015F0002CF00AC0EDFF09C0EDFF08C0EDFF07C0E9
:10160000EFFFFB0EDBCF14F0FC0EDBCF15F0FD0E71
:10161000DBCF16F0FE0EDBCF17F00C6A0D6A200E42
:101620000E6E410E0F6E14C007F015C008F016C004
:1016300009F017C00AF00DEC2FF0010A13E0FB0EC1
:10164000DB6AFC0EDB6A800EF36EFD0EF3CFDBFF70
:101650003F0EF36EFE0EF3CFDBFF020EDB2A030E0E
:1016600001E3DB2A020EDBCF14F0030EDBCF15F013
:101670000001800E15145FE0F90EDBCFE9FFDB2AD5
:10168000FA0EDBCFEAFF01E3DB2A300EEF6EF90E34
:10169000DBCFE9FFDB2AFA0EDBCFEAFF01E3DB2A2F
:1016A0002E0EEF6E080EDBCF14F0090EDBCF15F017
:1016B000800E151414E0020EDBCF16F0030EDBCF04
:1016C00017F0080EDB50165C146E090EDB5017582D
:1016D000156E020E14C0DBFF030E15C0DBFF040EF7
:1016E000DB68050EDB68040EDBCF14F0050EDBCFE4
:1016F00015F0020EDBCF16F0030EDBCF17F01750FC
:101700001518E8AE02D0153404D01450165C1550EC
:10171000175811E2F90EDBCFE9FFDB2AFA0EDBCF17
:10172000EAFF01E3DB2A300EEF6E040EDB06050E46
:1017300001E2DB06D8D7040EDB6A050EDB6A040E75
:10174000DBCF14F0050EDBCF15F0080EDBCF16F063
:10175000090EDBCF17F015501718E8AE02D017347A
:1017600004D01650145C1750155801E3ACD0FB0E92
:10177000DBCF07F0FC0EDBCF08F0FD0EDBCF09F06E
:10178000FE0EDBCF0AF09EEC2EF0060E08C0DBFF4B
:10179000070E09C0DBFF300EE76E060EDBCF14F03C
:1017A000070EDBCF15F0E7501426000E1522F90EB8
:1017B000DBCFE9FFDB2AFA0EDBCFEAFF01E3DB2A0E
:1017C00014C0EFFF040EDBCF14F0050EDBCF15F0D5
:1017D000020EDB50141803E1030EDB5015180BE169
:1017E000F90EDBCFE9FFDB2AFA0EDBCFEAFF01E3DC
:1017F000DB2A2E0EEF6E060EDBCF08F0070EDBCFD6
:1018000009F0CCEC2CF00A0E07C0DBFF0B0E08C071
:10181000DBFF0C0E09C0DBFF0D0E0AC0DBFF07C0AB
:1018200014F008C015F009C016F00AC017F0D9501E
:10183000FB0FE96EFF0EDA20EA6EEECF07F0EECF77
:1018400008F0EECF09F0EFCF0AF014C00CF015C08D
:101850000DF016C00EF017C00FF0FAEC2CF00AC015
:10186000EDFF09C0EDFF08C0EDFF07C0EFFF146AF0
:10187000156A200E166E410E176ED950FB0FE96ED9
:10188000FF0EDA20EA6EEECF07F0EECF08F0EECFD3
:1018900009F0EFCF0AF014C00CF015C00DF016C01F
:1018A0000EF017C00FF0E4EC2DF00AC0EDFF09C0F8
:1018B000EDFF08C0EDFF07C0EFFF040EDB2A050EA9
:1018C00001E3DB2A3CD7F90EDBCFE9FFFA0EDBCFD1
:1018D000EAFFEF6A0E0EE15C02E2E16AE552E16EB8
:1018E000E552E7CFD9FF1200D9CFE6FFE1CFD9FF0C
:1018F000060EE1260701CF9DFB0EDBCF07F0FC0EA5
:10190000DBCF08F0FD0EDBCF09F0FE0EDBCF0AF0D7
:10191000CDEC2EF006C0DEFF07C0DEFF08C0DEFF04
:1019200009C0DDFFDD52DD52F90EDBCF08F0FA0E03
:10193000DBCF09F0CCEC2CF007C014F008C015F098
:1019400009C016F00AC017F0FB0EDBCF1CF0FC0E2E
:10195000DBCF1DF0FD0EDBCF1EF0FE0EDBCF1FF048
:10196000D9CFE9FFDACFEAFFEECF24F0EECF25F0B2
:10197000EECF26F0EFCF27F024C006F025C007F009
:1019800026C008F027C009F0E1EC2CF007C020F0D9
:1019900008C021F009C022F00AC023F020C00CF0DA
:1019A00021C00DF022C00EF023C00FF01CC007F0C4
:1019B0001DC008F01EC009F01FC00AF0FAEC2CF0A0
:1019C00007C018F008C019F009C01AF00AC01BF0CF
:1019D00018C00CF019C00DF01AC00EF01BC00FF0AB
:1019E00014C007F015C008F016C009F017C00AF0BF
:1019F000E4EC2DF09EEC2EF0040E08C0DBFF050E8B
:101A000009C0DBFFD90EE66E080EE66ED9CFE9FFFE
:101A1000DACFEAFFEECFE6FFEECFE6FFEECFE6FF4E
:101A2000EFCFE6FFEAEC34F0146E060EE15E1450E0
:101A30000701CFAF09D0D90EE66E080EE66EADEC09
:101A400000F0E552E5520CD0D90EE66E080EE66EB7
:101A50005CEC06F0E552E552F3CF16F7F4CF17F73A
:101A60000701CFAF06D02E0EE66E6BEC00F0E5520C
:101A700005D02E0EE66E93EC06F0E552E66A040EF3
:101A8000DBCFE6FF050EDBCFE6FF2DEC08F0E552DD
:101A9000E552E552060EE15C02E2E16AE552E16ED2
:101AA000E552E7CFD9FF1200D9CFE6FFE1CFD9FF4A
:101AB000E652800EDF6EDF50000813E2FE0EDB50B0
:101AC000DF1406E0310EE66E93EC06F0E55205D029
:101AD000300EE66E93EC06F0E552DF407F0BDF6ED2
:101AE000EAD7E552E552E7CFD9FF1200D9CFE6FF9A
:101AF000E1CFD9FF020EE126010EDB6AFE0EDB50BC
:101B0000F00BE8380F0B300FDF6EDF50390803E2BF
:101B1000070EDF24DF6EFE0EDB500F0B300FE76E7B
:101B2000010EE7CFDBFFDB5039080AE2070E146E27
:101B3000010EDBCFE7FF1450E726010EE7CFDBFFF6
:101B40000701CFBF11D0DFCFE6FF93EC06F0E552DF
:101B5000010EDBCFE6FF93EC06F0E552680EE66E71
:101B600093EC06F0E55210D0DFCFE6FF6BEC00F00F
:101B7000E552010EDBCFE6FF6BEC00F0E552680E9C
:101B8000E66E6BEC00F0E552020EE15C02E2E16A07
:101B9000E552E16EE552E7CFD9FF1200D9CFE6FF5B
:101BA000E1CFD9FFFB0EDBCF07F0FC0EDBCF08F057
:101BB000FD0EDBCF09F0FE0EDBCF0AF00A34000E7B
:101BC0000A1809E6D880000E0754000E0854000ECB
:101BD0000954000E0A540CE2D950FB0FE96EFF0EB7
:101BE000DA20EA6EEE06000EEE5AEE5AEE5ADAD718
:101BF000E552E7CFD9FF1200D9CFE6FFE1CFD9FFF9
:101C0000020EE126DE6ADD6ADECF14F0DDCF15F0CC
:101C1000FE0EDB50000115AE02D0D89003D0145C4C
:101C2000000E15580AE2200EE66E93EC06F0E5521F
:101C3000DF2A010E01E3DB2AE7D7020EE15C02E2B4
:101C4000E16AE552E16EE552E7CFD9FF12000F01DC
:101C5000426B428F428B42890901D90E296F080ECF
:101C60002A6F150E146E720E156E166A14C0E6FFFA
:101C700015C0E6FF16C0E6FF29C9E6FF2AC9E6FF40
:101C8000ACEC39F0176E050EE15E17500701CFAFCF
:101C90000ED0020EE66EEBEC00F0E55229C9E6FF2D
:101CA0002AC9E6FFADEC00F0E552E5520ED029C995
:101CB000E6FF2AC9E6FF5CEC06F0E552E552F3CFF9
:101CC00016F7F4CF17F7A3EC06F0E80EE66E030E56
:101CD000E66EE66AE66A62DFE552E552E552E552F3
:101CE0000F01418F419D418B418741954191406B4F
:101CF00012000F013D93799E7998C90E796E3D953A
:101D0000789E7898DD0E786E778A778877967794C4
:101D100077927790A09CA09AA28CA28A1200806AE7
:101D20000F01386B38813883388538870F0E926EF3
:101D30008168396B030E936E020E616EF19E8268AC
:101D40003A6B800E946E948E826A836A3B6BBF0EF0
:101D5000956E846A3C6B966A606A1200C280C19E6E
:101D6000C08EC08AC088C096C082C094C090C19600
:101D7000C194C192C1901200D9CFE6FFE1CFD9FF43
:101D8000020EE126FD0EDBCF14F0FE0EDBCF15F0C8
:101D9000D89014361536D89014361536010E142402
:101DA000C26E0A0EE66E91EC3BF0E552B3EC3BF0EE
:101DB000AEEC3BF0000901E0FBD79CEC3BF0F3CF2D
:101DC000DEFFF4CFDDFFDECF14F0DDCF15F014C061
:101DD000F3FF15C0F4FF020EE15C03E200D0E16AFC
:101DE000E552E16EE552E7CFD9FF1200CD9ECD9CC2
:101DF000CD8ACD88CD96CD94CD82CD90CC9ECC9AF7
:101E0000CC92CC909F80D08E9D90DB0EE66E0B0E18
:101E1000E66EEEEC3AF0E552E5529E90F28CCD90F3
:101E2000F28EF28C0701D56BD66B1200D9CFE6FF8C
:101E3000E1CFD9FF020EE126DE6ADD6AFB0EDBCFC1
:101E4000F6FFDB2AFC0EDBCFF7FF01E3DB2A0800FD
:101E5000F550E66EFD0EDBCFE9FFDB2AFE0EDBCF91
:101E6000EAFF01E3DB2AE552E750EF6EDF2A010EBD
:101E700001E3DB2ADECF14F0DDCF15F0D89015504A
:101E800004E6000E145C010E1558D8E3020EE15C66
:101E900002E2E16AE552E16EE552E7CFD9FF1200B6
:101EA000D9CFE6FFE1CFD9FF020EE126DE6ADD6A77
:101EB000FB0EDBCFF6FFDB2AFC0EDBCFF7FF01E3E7
:101EC000DB2A0800F550E66EFF0EE76EFD0EDBCF55
:101ED00014F0FE0EDBCF15F0E7501426000E15228D
:101EE000DE50145CE96EDD501558EA6EE552E7509D
:101EF000EF6EDF2A010E01E3DB2ADECF14F0DDCF27
:101F000015F0D890155004E6000E145C010E15581B
:101F1000CFE3020EE15C02E2E16AE552E16EE552D6
:101F2000E7CFD9FF1200D9CFE6FFE1CFD9FFFB0EF3
:101F3000DBCF14F0FC0EDBCF15F0FD0EDBCF16F07F
:101F4000FE0EDBCF17F014C006F015C007F016C068
:101F500008F017C009F0E1EC2CF007C068F708C0E2
:101F600069F709C06AF70AC06BF7BC0EF66E640E1B
:101F7000F76E0900F5CF6CF70900F5CF6DF7090092
:101F8000F5CF6EF70800F5CF6FF76CC70CF06DC793
:101F90000DF06EC70EF06FC70FF068C707F069C786
:101FA00008F06AC709F06BC70AF091EC2DF007C082
:101FB00064F708C065F709C066F70AC067F764C729
:101FC000E6FF65C7E6FF66C7E6FF67C7E6FF0BECFF
:101FD00038F0E552E552E552E55206C014F007C06C
:101FE00015F008C016F009C017F014C007F015C0AE
:101FF00008F016C009F017C00AF0CDEC2EF006C0AC
:10200000C7F707C0C8F708C0C9F709C0CAF7070172
:10201000CF8F020EE66EEBEC00F0E5520901D90E0F
:10202000296F080E2A6F010EE66E29C9E6FF2AC93C
:10203000E6FF68C7E6FF69C7E6FF6AC7E6FF6BC74A
:10204000E6FF27EC09F0146E070EE15E145029C973
:10205000E6FF2AC9E6FFC5EC39F0E552E552F3CFB9
:1020600016F7F4CF17F70701070ED8801657000EA2
:102070001757060EE66E020EE66ECEEC00F0E55245
:10208000E552070116C714F017C715F01607000E22
:10209000175BD8801454000E155406E2200EE66E2D
:1020A0006BEC00F0E552EDD729C9E6FF2AC9E6FF3F
:1020B000ADEC00F0E552E552200EE66E6BEC00F060
:1020C000E552480EE66E6BEC00F0E5527A0EE66ED5
:1020D0006BEC00F0E5520701CF9F29C9E6FF2AC942
:1020E000E6FF5CEC06F0E552E552F3CF16F7F4CFCD
:1020F00017F7480EE66E93EC06F0E5527A0EE66EA0
:1021000093EC06F0E552A3EC06F00701CF8FC7C7AA
:10211000E2F7C8C7E1F7C9C7E0F7C26BC36BC46B8E
:10212000C56BE552E7CFD9FF12000701600E046FBF
:10213000000E056F04C702F705C703F7D96BDA6B0A
:10214000116B076B12000701CF8F010EE66EEBECEF
:1021500000F0E552080EE66EE66A92EC07F0E552F2
:10216000E552020EE66EEBEC00F0E552070EE66E6D
:10217000020EE66ECEEC00F0E552E55220C708F004
:1021800021C709F0CAEC2CF007C018F008C019F0FC
:1021900009C01AF00AC01BF00C6A0D6AC80E0E6E58
:1021A000420E0F6E18C007F019C008F01AC009F0EF
:1021B0001BC00AF0E4EC2DF007C014F008C015F0C5
:1021C00009C016F00AC017F00C6A0D6A800E0E6E78
:1021D000440E0F6E14C007F015C008F016C009F0C9
:1021E00017C00AF091EC2DF007C070F708C071F726
:1021F00009C072F70AC073F7020EE66E29C9E6FF3E
:102200002AC9E6FF70C7E6FF71C7E6FF72C7E6FF9F
:1022100073C7E6FF27EC09F0146E070EE15E145059
:1022200029C9E6FF2AC9E6FFADEC00F0E552E55208
:102230000701126B136B500EE66EC30EE66EE66A74
:10224000E66AACDCE552E552E552E552060E0701BE
:10225000986F996BFE0EE66E030EE66E020EE66E4A
:10226000E66A20C7E6FF21C7E6FF87EC1AF0146E86
:10227000060EE15E1450F3CF20F7F4CF21F70701EB
:10228000CF9F070EE66EE66A92EC07F0E552E55244
:1022900029C9E6FF2AC9E6FF5CEC06F0E552E552E3
:1022A000F3CF16F7F4CF17F7A3EC06F00701CF8FA3
:1022B000060E986F996B1200010EE66EEBEC00F0C3
:1022C000E5520A0EE66EE66A92EC07F0E552E55238
:1022D000020EE66EEBEC00F0E5523CC906F03DC99B
:1022E00007F03EC908F03FC909F0E1EC2CF007C047
:1022F00068F708C069F709C06AF70AC06BF70901F7
:10230000D90E296F080E2A6F010EE66E29C9E6FF65
:102310002AC9E6FF68C7E6FF69C7E6FF6AC7E6FFA6
:102320006BC7E6FF27EC09F0146E070EE15E145050
:1023300029C9E6FF2AC9E6FFC5EC39F0E552E552A6
:10234000F3CF16F7F4CF17F70701070ED88016570B
:10235000000E1757060EE66E020EE66ECEEC00F08B
:10236000E552E552070116C714F017C715F0160716
:10237000000E175BD8801454000E155406E2200E90
:10238000E66E6BEC00F0E552EDD729C9E6FF2AC9ED
:10239000E6FFADEC00F0E552E552200EE66E6BEC88
:1023A00000F0E552480EE66E6BEC00F0E5527A0E56
:1023B000E66E6BEC00F0E552500EE66EC30EE66E74
:1023C000E66AE66ACEEC0DF0E552E552E552E552DA
:1023D000A80EE66E610EE66EE66AE66A010EE66E2D
:1023E000E66AE66AE66A3CC9E6FF3DC9E6FF3EC921
:1023F000E6FF3FC9E6FF7AEC17F0146E0C0EE15EC3
:10240000145006C03CF907C03DF908C03EF909C0A8
:102410003FF93CC9E6FF3DC9E6FF3EC9E6FF3FC9BB
:10242000E6FF81DDE552E552E552E5520701CF8F27
:10243000020EE66EEBEC00F0E5523CC906F03DC939
:1024400007F03EC908F03FC909F0E1EC2CF007C0E5
:1024500068F708C069F709C06AF70AC06BF7090195
:10246000D90E296F080E2A6F010EE66E29C9E6FF04
:102470002AC9E6FF68C7E6FF69C7E6FF6AC7E6FF45
:102480006BC7E6FF27EC09F0146E070EE15E1450EF
:1024900029C9E6FF2AC9E6FFC5EC39F0E552E55245
:1024A000F3CF16F7F4CF17F70701070ED8801657AA
:1024B000000E1757060EE66E020EE66ECEEC00F02A
:1024C000E552E552070116C714F017C715F01607B5
:1024D000000E175BD8801454000E155406E2200E2F
:1024E000E66E6BEC00F0E552EDD729C9E6FF2AC98C
:1024F000E6FFADEC00F0E552E552200EE66E6BEC27
:1025000000F0E552480EE66E6BEC00F0E5527A0EF4
:10251000E66E6BEC00F0E552500EE66EC30EE66E12
:10252000E66AE66ACEEC0DF0E552E552E552E55278
:102530001200010EE66EEBEC00F0E552090EE66EBD
:10254000E66A92EC07F0E552E5521EC7E9FF1FC7A5
:10255000EAFFD890E936EA36FF0EE926070EEA22AE
:10256000EECF3CF9EFCF3DF909013E6B3F6B020E18
:10257000E66EEBEC00F0E552020EE66EE66ECEEC97
:1025800000F0E552E5521EC714F01FC715F00A0E01
:102590000D6E0E6A14C008F015C009F051EC2EF053
:1025A00008C014F009C015F0300E1424E66E6BEC70
:1025B00000F0E5521EC714F01FC715F00A0E0D6E8D
:1025C0000E6A14C008F015C009F051EC2EF004C0DA
:1025D00014F005C015F0300E1424E66E6BEC00F01C
:1025E000E552200EE66E6BEC00F0E552200EE66E32
:1025F0006BEC00F0E552080EE66E020EE66ECEECD5
:1026000000F0E552E5523CC906F03DC907F03EC96D
:1026100008F03FC909F0E1EC2CF007C068F708C0EA
:1026200069F709C06AF70AC06BF7010EE66E29C99F
:10263000E6FF2AC9E6FF68C7E6FF69C7E6FF6AC783
:10264000E6FF6BC7E6FF27EC09F0146E070EE15EAC
:10265000145029C9E6FF2AC9E6FFADEC00F0E552A7
:10266000E552200EE66E6BEC00F0E552480EE66E89
:102670006BEC00F0E5527A0EE66E6BEC00F0E55282
:102680000701126B136B000EE66EE66ABCEC0EF0EF
:10269000E552E552F3CF9EF7F4CF9FF70701FA0E0C
:1026A0009E5D000E9F5909E3EE0ED8809E55020EE6
:1026B0009F5503E38D848D828D80EE0ED8809E55CC
:1026C000020E9F5510E28D948D828D801E2B000E80
:1026D0001F231F3504E21E513F08000E1F5503E261
:1026E000010E1E6F1F6BFA0E9E5D000E9F5912E2C7
:1026F0008D848D828D901E07000E1F5B010E1FAF13
:1027000002D0D89003D01E5D000E1F5903E23F0E89
:102710001E6F1F6B1EC7E9FF1FC7EAFFD890E9367F
:10272000EA36FF0EE926070EEA22EECF3CF9EFCF9C
:102730003DF909013E6B3F6B020EE66EEBEC00F0DB
:10274000E5521EC714F01FC715F00A0E0D6E0E6A73
:1027500014C008F015C009F051EC2EF008C014F0B8
:1027600009C015F0300E1424E66E6BEC00F0E55253
:102770001EC714F01FC715F00A0E0D6E0E6A14C0A6
:1027800008F015C009F051EC2EF004C014F005C09B
:1027900015F0300E1424E66E6BEC00F0E552200EBE
:1027A000E66E6BEC00F0E552200EE66E6BEC00F08E
:1027B000E552060EE66E020EE66ECEEC00F0E55235
:1027C000E5523CC906F03DC907F03EC908F03FC9D3
:1027D00009F0E1EC2CF007C068F708C069F709C000
:1027E0006AF70AC06BF7010EE66E29C9E6FF2AC92F
:1027F000E6FF68C7E6FF69C7E6FF6AC7E6FF6BC783
:10280000E6FF27EC09F0146E070EE15E145029C9AB
:10281000E6FF2AC9E6FFADEC00F0E552E552200ED6
:10282000E66E6BEC00F0E552480EE66E6BEC00F0E5
:10283000E5527A0EE66E6BEC00F0E552A00EE66E05
:10284000860EE66E010EE66EE66ACEEC0DF0E552FF
:10285000E552E552E55281B016D7880EE66E130EAA
:10286000E66EE66AE66ACEEC0DF0E552E552E55218
:10287000E55281A0FED78D848D828D8012000701E4
:10288000CF9F010EE66EE66A92EC07F0E552E55244
:102890000701CF8F010EE66EEBEC00F0E552010E62
:1028A000E66EE66A92EC07F0E552E5520701126B1C
:1028B000136B000E125D010E135946E2BC0E122579
:1028C000F66E600E1321F76E0800F5CF18F018C0F1
:1028D00009F0B9EC2CF007C014F008C015F009C0DD
:1028E00016F00AC017F00C6A0D6A0E6A410E0F6EE0
:1028F00014C007F015C008F016C009F017C00AF0A0
:1029000091EC2DF007C074F708C075F709C076F791
:102910000AC077F774C707F075C708F076C709F0E3
:1029200077C70AF077EC2EF00950E66E000E07012B
:102930001225E96E060E1321EA6EE552E750EF6E9E
:10294000122B000E1323B5D712000701CF9F020EE2
:10295000E66EE66A92EC07F0E552E5520701CF8F8A
:10296000010EE66EEBEC00F0E552020EE66EE66A52
:1029700092EC07F0E552E5520701126B136B800EE3
:10298000125D000E13590CE2000E1225E96E060EC0
:102990001321EA6E1F0EEF6E122B000E1323EFD7DA
:1029A000800E126F136B000E125D010E13590BE2B5
:1029B000000E1225E96E060E1321EA6EEF6A122B45
:1029C000000E1323F0D712000701CF9F030EE66E0F
:1029D000E66A92EC07F0E552E5520701CF8F010E4F
:1029E000E66EEBEC00F0E552030EE66EE66A92EC62
:1029F00007F0E552E5520701126B136B800E125D72
:102A0000000E135940E212C708F013C709F0CAECD0
:102A10002CF007C014F008C015F009C016F00AC069
:102A200017F00C6A0D6A800E0E6E400E0F6E14C009
:102A300007F015C008F016C009F017C00AF091ECB5
:102A40002DF007C074F708C075F709C076F70AC003
:102A500077F774C707F075C708F076C709F077C72E
:102A60000AF077EC2EF00950E66E000E07011225F1
:102A7000E96E060E1321EA6EE552E750EF6E122B57
:102A8000000E1323BBD7800E126F136B000E125D66
:102A9000010E135949E212C718F013C719F0FF0EBF
:102AA000D8801856000E195618C008F019C009F041
:102AB000CAEC2CF007C014F008C015F009C016F0DD
:102AC0000AC017F00C6A0D6A800E0E6E400E0F6E73
:102AD00014C007F015C008F016C009F017C00AF0BE
:102AE00091EC2DF007C074F708C075F709C076F7B0
:102AF0000AC077F774C707F075C708F076C709F002
:102B000077C70AF077EC2EF00950E66E000E070149
:102B10001225E96E060E1321EA6EE552E750EF6EBC
:102B2000122B000E1323B2D712000701CF9F040E01
:102B3000E66EE66A92EC07F0E552E5520701CF8FA8
:102B4000010EE66EEBEC00F0E552040EE66EE66A6E
:102B500092EC07F0E552E5520701126B136B000E81
:102B6000125D010E13593FE212C708F013C709F0B6
:102B7000CAEC2CF007C014F008C015F009C016F01C
:102B80000AC017F00C6A0D6A0E6A410E0F6E14C06F
:102B900007F015C008F016C009F017C00AF091EC54
:102BA0002DF007C074F708C075F709C076F70AC0A2
:102BB00077F774C707F075C708F076C709F077C7CD
:102BC0000AF077EC2EF00950E66E000E0701122590
:102BD000E96E060E1321EA6EE552E750EF6E122BF6
:102BE000000E1323BCD712000701CF9F050EE66E1F
:102BF000E66A92EC07F0E552E5520701CF8F010E2D
:102C0000E66EEBEC00F0E552050EE66EE66A92EC3D
:102C100007F0E552E5520701126B136B000E125DCF
:102C2000010E135948E212C718F013C719F0FF0E2E
:102C3000D8801856000E195618C008F019C009F0AF
:102C4000CAEC2CF007C014F008C015F009C016F04B
:102C50000AC017F00C6A0D6A0E6A410E0F6E14C09E
:102C600007F015C008F016C009F017C00AF091EC83
:102C70002DF007C074F708C075F709C076F70AC0D1
:102C800077F774C707F075C708F076C709F077C7FC
:102C90000AF077EC2EF00950E66E000E07011225BF
:102CA000E96E060E1321EA6EE552E750EF6E122B25
:102CB000000E1323B3D71200D9CFE6FFE1CFD9FF1F
:102CC000020EE12620C714F021C715F0D890153266
:102CD0001432D8901532143214C0DEFF15C0DDFF57
:102CE0000701CF9F060EE66EE66A92EC07F0E5520A
:102CF000E5520701CF8F010EE66EEBEC00F0E552D6
:102D0000060EE66EE66A92EC07F0E552E552D9CF80
:102D1000E9FFDACFEAFF000ED880EE54000EED5442
:102D200035E2DECF14F0DDCF15F0FF0E145C000E9F
:102D300015582CE20701126B136BDECF14F0DDCFB8
:102D400015F01450125D155013590CE2000E1225A7
:102D5000E96E060E1321EA6E1F0EEF6E122B000EA7
:102D60001323EBD7DECF12F7DDCF13F7000E125D82
:102D7000010E13590BE2000E1225E96E060E132107
:102D8000EA6EEF6A122B000E1323F0D7020EE15CFD
:102D900002E2E16AE552E16EE552E7CFD9FF1200A7
:102DA000200EE66E6BEC00F0E552060EE66E020EAB
:102DB000E66ECEEC00F0E552E552A6C706F0A7C7D6
:102DC00007F0A8C708F0A9C709F0E1EC2CF007C08C
:102DD00074F708C075F709C076F70AC077F70901DC
:102DE000D90E296F080E2A6F010EE66E29C9E6FF7B
:102DF0002AC9E6FF74C7E6FF75C7E6FF76C7E6FF98
:102E000077C7E6FF27EC09F0146E070EE15E145059
:102E10000701070E961901E197511BE1030EE66EBB
:102E2000020EE66ECEEC00F0E552E55229C9E6FF4F
:102E30002AC9E6FFC5EC39F0E552E552F3CF14F7A5
:102E4000F4CF15F707010A0ED8801457000E155756
:102E50001AD029C9E6FF2AC9E6FFC5EC39F0E552C8
:102E6000E552F3CF14F7F4CF15F70701070ED8801A
:102E70001457000E1557060EE66E020EE66ECEECE7
:102E800000F0E552E552070114C714F015C715F01C
:102E90001407000E155BD8801454000E155406E27A
:102EA000200EE66E6BEC00F0E552EDD729C9E6FF87
:102EB0002AC9E6FFADEC00F0E552E552200EE66EC1
:102EC0006BEC00F0E552480EE66E6BEC00F0E5525C
:102ED0007A0EE66E6BEC00F0E552880EE66E130E8D
:102EE000E66EE66AE66ACEEC0DF0E552E552E55292
:102EF000E5521200D9CFE6FFE1CFD9FF080EE12657
:102F0000FB0EDBCFA6F7FC0EDBCFA7F7FD0EDBCF6A
:102F1000A8F7FE0EDBCFA9F781A0FED7060EDB6A6D
:102F2000070EDB6ACD909E900701D16BD26B000E2D
:102F3000E66EE66ABCEC0EF0E552E552F3CFDEFF3A
:102F4000F4CFDDFFD00EE66E070EE66EE66AE66AA7
:102F5000CEEC0DF0E552E552E552E552D9CFE9FF4E
:102F6000DACFEAFFEE0ED880EE54020EED541CE3E9
:102F7000DECF14F0DDCF15F0FA0E145C000E1558FC
:102F800013E38D848D808D92E66A020EE66ECEECA0
:102F900000F0E552E5523D0EE66E6BEC00F0E552B6
:102FA000FFDE0701D16BD26BD9CFE9FFDACFEAFFA1
:102FB000EE0ED880EE54020EED5401E3DDD08D9478
:102FC0008D828D800701D16BD26BD9CFE9FFDACF2B
:102FD000EAFFEE0ED880EE54020EED5401E3CCD0A1
:102FE000000EE66EE66ABCEC0EF0E552E552F3CF59
:102FF000DEFFF4CFDDFF0701D12B000ED223D1C7B6
:1030000014F0D2C715F0030ED89015321432E8042C
:10301000FBE1060E14C0DBFF070E15C0DBFFD95025
:10302000060FE96EDACFEAFF0A0ED880EE54000EE2
:10303000ED5407E20A0EF36E060EF3CFDBFF070E28
:10304000DB6A0701070E961901E197511DE1060E93
:10305000DBCFE9FF070EDBCFEAFF020ED890E9369F
:10306000EA36E806FBE1AB0EE926080EEA22020E7C
:10307000EECFDBFF030EEECFDBFF040EEECFDBFF68
:10308000050EEECFDBFF1ED0060EDBCFE9FF070EED
:10309000DBCFEAFF010ED890E936EA36E806FBE11D
:1030A000950EE926080EEA22EECF14F0EFCF15F0C8
:1030B000020E14C0DBFF030E15C0DBFF040EDB6A3B
:1030C000050EDB6AD950020FE96EDACFEAFF07017D
:1030D000A651EE24146EA751EE20156EA851EE20D5
:1030E000166EA951EE20176EF30EDBCF07F0F40E2B
:1030F000DBCF08F0F50EDBCF09F0F60EDBCF0AF0E0
:1031000017500A18E8AE02D00A3408D00750145CF1
:1031100008501558095016580A50175812E2D9503D
:10312000020FE96EDACFEAFFA651EE24A66FA7518F
:10313000EE20A76FA851EE20A86FA951EE20A96F2D
:103140000CD0F30EDBCFA6F7F40EDBCFA7F7F50E0E
:10315000DBCFA8F7F60EDBCFA9F7CF8FE66A020E1A
:10316000E66ECEEC00F0E552E5523E0EE66E6BECFC
:1031700000F0E55215DE29D7DECF14F0DDCF15F0D3
:10318000FA0E145C000E155801E3D6D08D848D82A2
:103190008D900701D16BD26BDECF14F0DDCF15F02F
:1031A000FA0E145C000E155801E3C6D00701D12BAE
:1031B000000ED223E66EE66ABCEC0EF0E552E55254
:1031C000F3CFDEFFF4CFDDFFD1C714F0D2C715F087
:1031D000030ED89015321432E804FBE1060E14C039
:1031E000DBFF070E15C0DBFFD950060FE96EDACF03
:1031F000EAFF0A0ED880EE54000EED5407E20A0EE4
:10320000F36E060EF3CFDBFF070EDB6A0701070E36
:10321000961901E197511DE1060EDBCFE9FF070E7C
:10322000DBCFEAFF020ED890E936EA36E806FBE18A
:10323000AB0EE926080EEA22020EEECFDBFF030EEC
:10324000EECFDBFF040EEECFDBFF050EEECFDBFF94
:103250001ED0060EDBCFE9FF070EDBCFEAFF010E23
:10326000D890E936EA36E806FBE1950EE926080E25
:10327000EA22EECF14F0EFCF15F0020E14C0DBFF00
:10328000030E15C0DBFF040EDB6A050EDB6AF70ECA
:10329000DBCF14F0F80EDBCF15F0F90EDBCF16F014
:1032A000FA0EDBCF17F0D950020FE96EDACFEAFF42
:1032B000EE501426EE501522EE501622EE50172234
:1032C00017500701A919E8AE02D0A93508D0A651B8
:1032D000145CA7511558A8511658A951175812E255
:1032E000D950020FE96EDACFEAFFEE50A65DA66F65
:1032F000EE50A759A76FEE50A859A86FEE50A959E4
:10330000A96F0CD0F70EDBCFA6F7F80EDBCFA7F72F
:10331000F90EDBCFA8F7FA0EDBCFA9F7E66A020EAB
:10332000E66ECEEC00F0E552E5523C0EE66E6BEC3C
:1033300000F0E55235DD30D781B0F0D5880EE66E6D
:10334000130EE66EE66AE66ACEEC0DF0E552E55243
:10335000E552E55281A0FED78D848D808D820701D4
:10336000CF9F0901D90E296F080E2A6FA6C706F054
:10337000A7C707F0A8C708F0A9C709F0E1EC2CF02F
:1033800007C074F708C075F709C076F70AC077F769
:10339000010EE66E29C9E6FF2AC9E6FF74C7E6FFFB
:1033A00075C7E6FF76C7E6FF77C7E6FF27EC09F0AB
:1033B000146E070EE15E145029C9E6FF2AC9E6FF24
:1033C0005CEC06F0E552E552F3CF14F0F4CF15F0C3
:1033D000166A176A15AE02D016681768020E14C076
:1033E000DBFF030E15C0DBFF040E16C0DBFF050E6E
:1033F00017C0DBFFA3EC06F00701CF8FA6C706F0CE
:10340000A7C707F0A8C708F0A9C709F0080EE15C34
:1034100003E200D0E16AE552E16EE552E7CFD9FF61
:1034200012000701CF8F200EE66E6BEC00F0E55224
:10343000070EE66E020EE66ECEEC00F0E552E552A7
:10344000A4C708F0A5C709F0CAEC2CF007C018F013
:1034500008C019F009C01AF00AC01BF00C6A0D6A06
:10346000C80E0E6E420E0F6E18C007F019C008F09D
:103470001AC009F01BC00AF0E4EC2DF007C014F0EC
:1034800008C015F009C016F00AC017F00C6A0D6AE2
:10349000800E0E6E440E0F6E14C007F015C008F0BB
:1034A00016C009F017C00AF091EC2DF007C070F7B4
:1034B00008C071F709C072F70AC073F7010EE66E13
:1034C00029C9E6FF2AC9E6FF70C7E6FF71C7E6FF14
:1034D00072C7E6FF73C7E6FF27EC09F0146E070E0C
:1034E000E15E145029C9E6FF2AC9E6FFADEC00F001
:1034F000E552E552100EE66E270EE66EE66AE66AC3
:10350000CEEC0DF0E552E552E552E5521200D9CF6E
:10351000E6FFE1CFD9FF040EE126FD0EDBCFA4F7D5
:10352000FE0EDBCFA5F7CD900701CF8F020EE66E22
:10353000EBEC00F0E5520701D16BD26B146B156B0D
:10354000000EE66EE66ABCEC0EF0E552E552F3CFF3
:10355000DEFFF4CFDDFFD00EE66E070EE66EE66A04
:10356000E66ACEEC0DF0E552E552E552E552D9CFD0
:10357000E9FFDACFEAFFEE0ED880EE54020EED54EA
:103580001EE3DECF14F0DDCF15F0FA0E145C000E52
:10359000155815E38D848D808D92E66A020EE66ED5
:1035A000CEEC00F0E552E5523D0EE66E6BEC00F01D
:1035B000E55237DF0701D16BD26B146B156BD9CF96
:1035C000E9FFDACFEAFFEE0ED880EE54020EED549A
:1035D00001E37ED00701D16BD26B8D948D828D80FB
:1035E000D9CFE9FFDACFEAFFEE0ED880EE54020E13
:1035F000ED546EE2000EE66EE66ABCEC0EF0E552AB
:10360000E552F3CFDEFFF4CFDDFF0701D12B000E33
:10361000D223D1C714F0D2C715F0030ED8901532BB
:103620001432E804FBE114C014F715C015F70701C4
:103630000A0ED8801455000E155503E20A0E146FB9
:10364000156B14C7E9FF15C7EAFF010ED890E936DC
:10365000EA36E806FBE17F0EE926080EEA22020EB2
:10366000EECFDBFF030EEDCFDBFF020EDB500701D9
:10367000A4250001146E030EDB500701A5210001F3
:10368000156EF90EDBCF16F0FA0EDBCF17F01650E1
:10369000145C1750155808E2020EDB500701A427EE
:1036A000030EDB50A52306D0F90EDBCFA4F7FA0EEC
:1036B000DBCFA5F7E66A020EE66ECEEC00F0E5522F
:1036C000E5523E0EE66E6BEC00F0E552AADE88D7BE
:1036D000DECF14F0DDCF15F0FA0E145C000E155895
:1036E00001E37ED00701D16BD26BDECF14F0DDCFCA
:1036F00015F0FA0E145C000E155872E28D848D825E
:103700008D900701D12B000ED223E66EE66ABCEC49
:103710000EF0E552E552F3CFDEFFF4CFDDFFD1C767
:1037200014F0D2C715F0030ED89015321432E80405
:10373000FBE114C014F715C015F707010A0ED88075
:103740001455000E155503E20A0E146F156B14C7BD
:10375000E9FF15C7EAFF010ED890E936EA36E80618
:10376000FBE17F0EE926080EEA22020EEECFDBFF18
:10377000030EEDCFDBFF020EDB500701A45D00015D
:10378000146E030EDB500701A5590001156EFB0EE8
:10379000DBCF16F0FC0EDBCF17F01450165C155083
:1037A000175808E2020EDB500701A45F030EDB503E
:1037B000A55B06D0FB0EDBCFA4F7FC0EDBCFA5F795
:1037C0000701CF8FE66A020EE66ECEEC00F0E552FE
:1037D000E5523E0EE66E6BEC00F0E55222DE85D738
:1037E00081B0A9D6880EE66E130EE66EE66AE66A2A
:1037F000CEEC0DF0E552E552E552E55281A0FED740
:103800008D848D808D820701CF9FA4C708F0A5C746
:1038100009F0CAEC2CF007C018F008C019F009C074
:103820001AF00AC01BF00C6A0D6AC80E0E6E420E2A
:103830000F6E18C007F019C008F01AC009F01BC0BD
:103840000AF0E4EC2DF007C014F008C015F009C030
:1038500016F00AC017F00C6A0D6A800E0E6E440E48
:103860000F6E14C007F015C008F016C009F017C09D
:103870000AF091EC2DF007C070F708C071F709C08D
:1038800072F70AC073F7020EE66E29C9E6FF2AC96D
:10389000E6FF70C7E6FF71C7E6FF72C7E6FF73C7B2
:1038A000E6FF27EC09F0146E070EE15E145029C9FB
:1038B000E6FF2AC9E6FF5CEC06F0E552E552020E8F
:1038C000F3CFDBFF030EF4CFDBFFA3EC06F0070121
:1038D000CF8FA4C7F3FFA5C7F4FF040EE15C03E29A
:1038E00000D0E16AE552E16EE552E7CFD9FF120060
:1038F000060E0701981901E1995129E0050E981962
:1039000001E1995121E0040E981901E1995119E062
:10391000030E981901E1995111E0020E981901E185
:10392000995109E0010E981901E1995101E012D075
:103930003FEC14F00FD0A5EC14F00CD0E4EC14F034
:1039400009D095EC15F006D0F4EC15F003D05CEC42
:1039500016F000D03CC9E6FF3DC9E6FF3EC9E6FFD0
:103960003FC9E6FF93EC0FF0E552E552E552E55210
:103970001200D9CFE6FFE1CFD9FF020EE126A09CCD
:10398000A09A0701CF8F010E9A1901E19B5119E10D
:10399000962B000E9723973504E296510708000EE8
:1039A000975503E2010E966F976B980EE66E3A0EEE
:1039B000E66EE66AE66ACEEC0DF0E552E552E552B7
:1039C000E5520701010E9C1901E19D5115E1960791
:1039D000000E975B9651971103E1070E966F976B58
:1039E000980EE66E3A0EE66EE66AE66ACEEC0DF0EA
:1039F000E552E552E552E552070E0701961901E13D
:103A0000975131E0060E961901E1975129E0050E14
:103A1000961901E1975121E0040E961901E19751A1
:103A200019E0030E961901E1975111E0020E961963
:103A300001E1975109E0010E961901E1975101E06A
:103A400015D03FEC14F012D0A5EC14F00FD0E4EC3C
:103A500014F00CD095EC15F009D0F4EC15F006D06C
:103A60005CEC16F003D0BDEC03F000D00701116B45
:103A7000146B156B010E9A1901E19B5103E19A6BCE
:103A80009B6BA19C010E9C1901E19D5103E19C6B74
:103A90009D6BA19A070E97AF02D0D89003D0965D88
:103AA000000E97590EE23CC9E6FF3DC9E6FF3EC94C
:103AB000E6FF3FC9E6FF93EC0FF0E552E552E55211
:103AC000E552A08CA08AF2929E90F2889D8A07010E
:103AD000CF9F100EE66E270EE66EE66AE66ACEEC23
:103AE0000DF0E552E552E552E55295EC10F0020E6C
:103AF000E15C02E2E16AE552E16EE552E7CFD9FF0F
:103B00001200F00EE66E490EE66E020EE66EE66AF2
:103B1000CEEC0DF0E552E552E552E5528FEC0EF099
:103B2000826A89988D848D828D800701D56BD66BD2
:103B3000D16BD26B600E046F000E056F04C702F7E5
:103B400005C703F70901D90E296F080E2A6F07016F
:103B5000C26BC36BC46BC56B560ECB6FCC6BCD6B9E
:103B6000CE6B010E8A6F8B6BD06BD08DD089D095C8
:103B7000D09BD091D0930F6B106B0D6B0E6BDD6BE8
:103B8000DE6BCF9F13EC06F00C0EE66E93EC06F0A6
:103B9000E552400EE66E0D0EE66E030EE66EE66A28
:103BA000CEEC0DF0E552E552E552E552A3EC06F0FD
:103BB000E5C714F0E6C715F0166A14C0E6FF15C095
:103BC000E6FF16C0E6FFD90EE66E080EE66EACEC18
:103BD00039F0176E050EE15E1750D90EE66E080E2D
:103BE000E66E5CEC06F0E552E552F3CF16F7F4CF43
:103BF00017F7A3EC06F0FDC714F0FEC715F0166A20
:103C000014C0E6FF15C0E6FF16C0E6FFD90EE66E4B
:103C1000080EE66EACEC39F0176E050EE15E17503B
:103C2000D90EE66E080EE66E5CEC06F0E552E55243
:103C3000F3CF16F7F4CF17F7A3EC06F0F9C714F09B
:103C4000FAC715F0166A14C0E6FF15C0E6FF16C0E5
:103C5000E6FFD90EE66E080EE66EACEC39F0176E94
:103C6000050EE15E1750D90EE66E080EE66E5CECAE
:103C700006F0E552E552F3CF16F7F4CF17F7FBC77E
:103C800014F0FCC715F0166A14C0E6FF15C0E6FF75
:103C900016C0E6FFD90EE66E080EE66EACEC39F003
:103CA000176E050EE15E1750D90EE66E080EE66E31
:103CB0005CEC06F0E552E552F3CF16F7F4CF17F7B8
:103CC000000EE66EE66A92EC07F0E552E5520D0E44
:103CD000E66EE66A92EC07F0E552E5520E0EE66EED
:103CE000E66A92EC07F0E552E552A3EC06F0F7C75E
:103CF00014F0F8C715F0166A14C0E6FF15C0E6FF09
:103D000016C0E6FFD90EE66E080EE66EACEC39F092
:103D1000176E050EE15E1750D90EE66E080EE66EC0
:103D20005CEC06F0E552E552F3CF16F7F4CF17F747
:103D3000BC0EF66E640EF76E0900F5CF6CF7090045
:103D4000F5CF6DF70900F5CF6EF70800F5CF6FF7E7
:103D5000060EE66E29C9E6FF2AC9E6FF6CC7E6FF34
:103D60006DC7E6FF6EC7E6FF6FC7E6FF27EC09F0F9
:103D7000146E070EE15E145029C9E6FF2AC9E6FF5A
:103D80005CEC06F0E552E552F3CF16F7F4CF17F7E7
:103D9000A3EC06F089980701CF8F0EEC00F0A00E7F
:103DA000E66E860EE66E010EE66EE66ACEEC0DF06D
:103DB000E552E552E552E552E66A010EE66ECEECBA
:103DC00000F0E552E552040EE66E720EE66E8AECE5
:103DD00000F0E552E552E66A020EE66ECEEC00F027
:103DE000E552E5520E0EE66EE66A92EC07F0E552F9
:103DF000E552900EE66ED00EE66E030EE66EE66AB3
:103E0000CEEC0DF0E552E552E552E5520701CF9FA9
:103E1000AEEC0EF00701DB6BDC6B126B136B000E6C
:103E2000125D010E135946E2BC0E1225F66E600EAD
:103E30001321F76E0800F5CF18F018C009F0B9EC9F
:103E40002CF007C014F008C015F009C016F00AC025
:103E500017F00C6A0D6A0E6A410E0F6E14C007F05F
:103E600015C008F016C009F017C00AF091EC2DF04B
:103E700007C074F708C075F709C076F70AC077F76E
:103E800074C707F075C708F076C709F077C70AF05E
:103E900077EC2EF00950E66E000E07011225E96E50
:103EA000060E1321EA6EE552E750EF6E122B000E5C
:103EB0001323B5D7010E966F976B986F996B0A0E07
:103EC0001E6F1F6B0901E80E3C6F030E3D6F3E6BCA
:103ED0003F6BF5C714F0F6C715F0166A14C0E6FF7D
:103EE00015C0E6FF16C0E6FFD90EE66E080EE66EB8
:103EF000ACEC39F0176E050EE15E1750D90EE66E88
:103F0000080EE66E5CEC06F0E552E552F3CF16F7CC
:103F1000F4CF17F70701C26BC36BC46BC56B3CC909
:103F200006F03DC907F03EC908F03FC909F0E1ECD1
:103F30002CF007C068F708C069F709C06AF70AC023
:103F40006BF76CC70CF06DC70DF06EC70EF06FC746
:103F50000FF068C707F069C708F06AC709F06BC7B8
:103F60000AF091EC2DF007C064F708C065F709C0AE
:103F700066F70AC067F764C7E6FF65C7E6FF66C76E
:103F8000E6FF67C7E6FF0BEC38F0E552E552E55275
:103F9000E55206C014F007C015F008C016F009C0BD
:103FA00017F014C007F015C008F016C009F017C0CC
:103FB0000AF0CDEC2EF006C0C7F707C0C8F708C05E
:103FC000C9F709C0CAF7D90EE66E080EE66EC7C774
:103FD000E6FFC8C7E6FFC9C7E6FFCAC7E6FFEAECC7
:103FE00034F0146E060EE15E1450D90EE66E080E23
:103FF000E66E5CEC06F0E552E552F3CF16F7F4CF2F
:1040000017F7090EE66E93EC06F0E552100EE66E19
:10401000270EE66EE66AE66ACEEC0DF0E552E55252
:10402000E552E5520701206B020E216FCF8F010E82
:10403000E66EEBEC00F0E552010EE66EE66A92ECFD
:1040400007F0E552E552020EE66EEBEC00F0E552A9
:10405000D90EE66E080EE66EADEC00F0E552E552C4
:104060003CC9E6FF3DC9E6FF3EC9E6FF3FC9E6FFA2
:1040700093EC0FF0E552E552E552E5520701CF9F70
:10408000A3EC06F079EC0EF0000EE66EE66ABCECEE
:104090000EF0E552E552F3CF9EF7F4CF9FF7010EF5
:1040A000E66EE66ABCEC0EF0E552E552F3CFA0F7FF
:1040B000F4CFA1F7EDC714F0EEC715F0166A14C0DF
:1040C000E6FF15C0E6FF16C0E6FFD90EE66E080E45
:1040D000E66EACEC39F0176E050EE15E1750030E7C
:1040E000E66EE66ABCEC0EF0E552E552F3CFA2F7BD
:1040F000F4CFA3F7A2C708F0A3C709F0CAEC2CF0CD
:1041000007C018F008C019F009C01AF00AC01BF067
:104110000C6A0D6AA00E0E6E400E0F6E18C007F0EE
:1041200019C008F01AC009F01BC00AF0E4EC2DF029
:1041300007C014F008C015F009C016F00AC017F047
:104140000C6A0D6A800E0E6E440E0F6E14C007F0DE
:1041500015C008F016C009F017C00AF091EC2DF058
:1041600007C074F708C075F709C076F70AC077F77B
:10417000A2C7E6FFA3C7E6FFA0C7E6FFA1C7E6FF09
:104180009EC7E6FF9FC7E6FF29C9E6FF2AC9E6FFEB
:10419000C20E146E710E156E166A14C0E6FF15C0BD
:1041A000E6FF16C0E6FFFE0EE66EE6685EEC39F04E
:1041B000176E0D0EE15E1750F3CF16F7F4CF17F719
:1041C000010EE66E29C9E6FF2AC9E6FF74C7E6FFBD
:1041D00075C7E6FF76C7E6FF77C7E6FF27EC09F06D
:1041E000146E070EE15E145029C9E6FF2AC9E6FFE6
:1041F0005CEC06F0E552E552F3CF16F7F4CF17F773
:10420000560EE66E93EC06F0E552A3EC06F00C0EAB
:10421000E66EE66A92EC07F0E552E55227EC0EF006
:10422000A3EC06F00701CF9F5F0E806F700E816FC9
:10423000090E826F420E836FEFC714F0F0C715F0BE
:10424000166A14C0E6FF15C0E6FF16C0E6FFD90ED9
:10425000E66E080EE66EACEC39F0176E050EE15E08
:104260001750D90EE66E080EE66E5CEC06F0E552CD
:10427000E552F3CF16F7F4CF17F7080EE66E29C90B
:10428000E6FF2AC9E6FF80C7E6FF81C7E6FF82C7CF
:10429000E6FF83C7E6FF27EC09F0146E070EE15E28
:1042A000145029C9E6FF2AC9E6FF5CEC06F0E55286
:1042B000E552F3CF16F7F4CF17F7A3EC06F007019A
:1042C000C66B946B956BE2EC02F007016F0ECB6F3F
:1042D0000C0ECC6F010ECD6FCE6BCBC7E6FF9CEC06
:1042E00003F0E552CCC7E6FF9CEC03F0E552CDC7E6
:1042F000E6FF9CEC03F0E552CEC7E6FF9CEC03F032
:10430000E552C6C7E6FF9CEC03F0E552010EE66EEF
:1043100091EC3BF0E5528B8A010EE66E91EC3BF09E
:10432000E5528B9A0701846B856BFA0E866F440EFB
:10433000876F0901D90E296F080E2A6F010EE66EEC
:1043400029C9E6FF2AC9E6FF84C7E6FF85C7E6FF5D
:1043500086C7E6FF87C7E6FF27EC09F0146E070E55
:10436000E15E145029C9E6FF2AC9E6FFCBC7E6FF84
:10437000CCC7E6FFCDC7E6FFCEC7E6FF880E146EBA
:10438000710E156E166A14C0E6FF15C0E6FF16C062
:10439000E6FFFE0EE66EE6685EEC39F0176E0B0E79
:1043A000E15E1750F3CF16F7F4CF17F7400EE66E25
:1043B000420EE66E0F0EE66EE66ACEEC0DF0E552AA
:1043C000E552E552E5520701800E846F960E856F27
:1043D000180E866F4B0E876F84C7E6FF85C7E6FF12
:1043E00086C7E6FF87C7E6FF3BEC03F0E552E552E0
:1043F000E552E5520901D90E296F080E2A6F010E08
:10440000E66E29C9E6FF2AC9E6FF84C7E6FF85C72D
:10441000E6FF86C7E6FF87C7E6FF27EC09F0146EC4
:10442000070EE15E145029C9E6FF2AC9E6FFCBC793
:10443000E6FFCCC7E6FFCDC7E6FFCEC7E6FF590EC5
:10444000146E710E156E166A14C0E6FF15C0E6FFF5
:1044500016C0E6FFFE0EE66EE6685EEC39F0176EFB
:104460000B0EE15E1750F3CF16F7F4CF17F7400E9F
:10447000E66E420EE66E0F0EE66EE66ACEEC0DF0CC
:10448000E552E552E552E5520701846B856B7A0EE1
:10449000866F440E876F84C7E6FF85C7E6FF86C731
:1044A000E6FF87C7E6FF3BEC03F0E552E552E55235
:1044B000E5520901D90E296F080E2A6F010EE66E2A
:1044C00029C9E6FF2AC9E6FF84C7E6FF85C7E6FFDC
:1044D00086C7E6FF87C7E6FF27EC09F0146E070ED4
:1044E000E15E145029C9E6FF2AC9E6FFCBC7E6FF03
:1044F000CCC7E6FFCDC7E6FFCEC7E6FF590E146E68
:10450000710E156E166A14C0E6FF15C0E6FF16C0E0
:10451000E6FFFE0EE66EE6685EEC39F0176E0B0EF7
:10452000E15E1750F3CF16F7F4CF17F7200EE66EC3
:104530004E0EE66EE66AE66ACEEC0DF0E552E55206
:10454000E552E5520701D16BD26BD36BD46BF6EC1D
:104550000EF00701146B156BD66A000EE66EE66A64
:104560000AEC3BF0E552E552040ED56EF29A9D6AD4
:10457000A06AA36A07019A6B9B6B9C6B9D6BA19CC5
:10458000A19A9D90CD90D09CD08EAB889D8AF288C8
:10459000A08AA08CF28CF28EF28CD0958988CF9F65
:1045A000D96BDA6B95EC10F007010451021902E1A6
:1045B0000551031901E19FD3ACEC06F00701076F29
:1045C000D92B000EDA23CF9F0751580A01E133D1CE
:1045D000080A01E1A1D0110A01E18DD0130A71E0AE
:1045E000160A55E0100A39E0170A1DE0100A01E02A
:1045F0003DD1010E966F976B3FEC14F03CC9E6FF7E
:104600003DC9E6FF3EC9E6FF3FC9E6FF93EC0FF068
:10461000E552E552E552E552050E0701926F936BA4
:1046200095EC10F023D1020E966F976BA5EC14F069
:104630003CC9E6FF3DC9E6FF3EC9E6FF3FC9E6FFCC
:1046400093EC0FF0E552E552E552E552050E0701F5
:10465000926F936B95EC10F009D1030E966F976BE8
:10466000E4EC14F03CC9E6FF3DC9E6FF3EC9E6FFB5
:104670003FC9E6FF93EC0FF0E552E552E552E552F3
:10468000050E0701926F936B95EC10F0EFD0040EBE
:10469000966F976B95EC15F03CC9E6FF3DC9E6FFB8
:1046A0003EC9E6FF3FC9E6FF93EC0FF0E552E55245
:1046B000E552E552050E0701926F936B95EC10F0F1
:1046C000D5D0050E966F976BF4EC15F03CC9E6FF5C
:1046D0003DC9E6FF3EC9E6FF3FC9E6FF93EC0FF098
:1046E000E552E552E552E552050E0701926F936BD4
:1046F00095EC10F0BBD0070E966F976B0B0EE66E25
:10470000E66A92EC07F0E552E55295EC10F0080EDF
:104710000701926F936BAAD0942B000E95239535C9
:1047200004E294511F08000E955502E2946B956BBC
:1047300094C714F095C715F0030ED89014361536AB
:10474000E804FBE114C0C6F794C708F095C709F068
:10475000CCEC2CF007C014F008C015F009C016F01E
:104760000AC017F00C6A0D6A340E0E6E410E0F6E01
:1047700014C007F015C008F016C009F017C00AF001
:10478000E4EC2DF007C074F708C075F709C076F7A0
:104790000AC077F7010EE66E29C9E6FF2AC9E6FFCF
:1047A00074C7E6FF75C7E6FF76C7E6FF77C7E6FF83
:1047B00027EC09F0146E070EE15E145029C9E6FFDC
:1047C0002AC9E6FF0701C651E66EE66A260E146E98
:1047D000710E156E166A14C0E6FF15C0E6FF16C00E
:1047E000E6FFFE0EE66EE6685EEC39F0176E090E27
:1047F000E15E1750F3CF16F7F4CF17F784C7E6FF43
:1048000085C7E6FF86C7E6FF87C7E6FF3BEC03F0F8
:10481000E552E552E552E552100EE66E270EE66EC1
:10482000E66AE66ACEEC0DF0E552E552E552E55255
:1048300095EC10F01BD0060E966F976BCF8FE66E3F
:10484000E66A92EC07F0E552E5520701CF9F060EAB
:10485000E66EE66A92EC07F0E552E55295EC10F050
:10486000040E0701926F936BCF8F00D0010E0701EA
:10487000156A9225146E935115221450D91902E12C
:104880001550DA1901E0FED10D0E075D01E0FAD1F5
:10489000DB6BDC6B126B136B9251125D93511359EE
:1048A00018E2600E1225E96E000E1321EA6EEF5039
:1048B000E66EE66A53EC3BF0E552E5520701DB5148
:1048C000F324DB6FDC51F420DC6F122B000E13237A
:1048D000E3D79251DB1902E19351DC1930E0F3C7C1
:1048E00014F0F4C715F0166A14C0E6FF15C0E6FF11
:1048F00016C0E6FFD90EE66E080EE66EACEC39F097
:10490000176E050EE15E1750D90EE66E080EE66EC4
:104910005CEC06F0E552E552F3CF16F7F4CF17F74B
:104920008998F00EE66E490EE66E020EE66EE66AB5
:10493000CEEC0DF0E552E552E552E552A0D1600E05
:104940009225E96E000E9321EA6EEF6A070E961922
:1049500001E1975101E1FCD0060E961901E1975152
:1049600045E0010E961901E1975115E0020E9619E6
:1049700001E1975110E0030E961901E197510BE008
:10498000040E961901E1975106E0050E961901E112
:10499000975101E074D1C76BC86BC96BCA6B600ECD
:1049A000E66E000EE66EA5EC33F0E552E55206C069
:1049B0003CF907C03DF908C03EF909C03FF93CC9C0
:1049C000E6FF3DC9E6FF3EC9E6FF3FC9E6FF93ECBF
:1049D0000FF0E552E552E552E55296C798F797C7B2
:1049E00099F778EC1CF00701116B49D1CF8F0001CA
:1049F000646B600EE66E000EE66E30EC33F0E5524E
:104A0000E552F3CF22F7F4CF23F70701FE0E225D24
:104A1000030E235901E39BD0020ED8802255000ECD
:104A2000235501E394D022C720F723C721F711ECC7
:104A30001AF0090EE66E93EC06F0E552600EE66E93
:104A4000000EE66E5CEC06F0E552E552F3CF16F789
:104A5000F4CF17F7200EE66E93EC06F0E5522D0E1C
:104A6000E66E93EC06F0E5523E0EE66E93EC06F031
:104A7000E552200EE66E93EC06F0E55220C708F0F2
:104A800021C709F0CAEC2CF007C018F008C019F0D3
:104A900009C01AF00AC01BF00C6A0D6AC80E0E6E2F
:104AA000420E0F6E18C007F019C008F01AC009F0C6
:104AB0001BC00AF0E4EC2DF007C014F008C015F09C
:104AC00009C016F00AC017F00C6A0D6A800E0E6E4F
:104AD000440E0F6E14C007F015C008F016C009F0A0
:104AE00017C00AF091EC2DF007C074F708C075F7F5
:104AF00009C076F70AC077F7010EE66E29C9E6FF0E
:104B00002AC9E6FF74C7E6FF75C7E6FF76C7E6FF6A
:104B100077C7E6FF27EC09F0146E070EE15E14502C
:104B200029C9E6FF2AC9E6FF5CEC06F0E552E5522A
:104B3000F3CF16F7F4CF17F7A3EC06F00701CF8FEA
:104B4000060E986F996B78EC1CF00701116B97D0EB
:104B50000001686B600EE66E000EE66EA5EC33F0A9
:104B6000E552E55206C0AEF707C0AFF708C0B0F790
:104B700009C0B1F7AEC706F0AFC707F0B0C708F07D
:104B8000B1C709F0DFEC2CF007C084F708C085F747
:104B900009C086F70AC087F784C7E6FF85C7E6FF26
:104BA00086C7E6FF87C7E6FF3BEC03F0E552E55218
:104BB000E552E5520701CF9F200EE66E93EC06F01A
:104BC000E552010EE66E29C9E6FF2AC9E6FF84C751
:104BD000E6FF85C7E6FF86C7E6FF87C7E6FF27EC47
:104BE00009F0146E070EE15E145029C9E6FF2AC9C8
:104BF000E6FFC5EC39F0E552E552F3CF14F7F4CFF8
:104C000015F707010A0ED8801457000E1557070133
:104C100014C714F015C715F01407000E155BD880E3
:104C20001454000E155406E2200EE66E6BEC00F0F4
:104C3000E552EDD7010EE66E29C9E6FF2AC9E6FF67
:104C400084C7E6FF85C7E6FF86C7E6FF87C7E6FF9E
:104C500027EC09F0146E070EE15E145029C9E6FF37
:104C60002AC9E6FF5CEC06F0E552E552F3CF16F7F1
:104C7000F4CF17F7A3EC06F00701116B00D0898879
:104C800095EC10F00701103504E20F510008000EFA
:104C9000105507E30E3504E20D510008000E0E55C5
:104CA00029E2E3C7E6FFE4C7E6FF23EC06F0E5529E
:104CB000E552F3CF0BF7F4CF0CF7E66A0FC7E6FF28
:104CC00010C7E6FF2DEC08F0E552E552E552090E5B
:104CD000E66E93EC06F0E552E66A0DC7E6FF0EC7F6
:104CE000E6FF2DEC08F0E552E552E552899895EC87
:104CF00010F001D08988A00EE66E860EE66E010ED9
:104D0000E66EE66ACEEC0DF0E552E552E552E5526C
:104D10009D8A0701146B156BC451EA6A000FE96E96
:104D2000060EEA22EFCF40FFC70EE96E070EEA6ECD
:104D3000C251EE24C26FC351EE20C36FC451EE20A6
:104D4000C46FC551EE20C56F1151E6E02DD412009D
:104D5000E4EC2BF0FB0EDBCFF3FFDB06F350000996
:104D60000AE032EC2CF0FA0E9DEC2CF0F3E1151C6D
:104D7000F1E1010E01D0000E13EF2CF0E4EC2BF06A
:104D80003B0EE12402E3E168E652E16E010EDB6ACC
:104D9000020EDB6AF90EDBCFF6FFFA0EDBCFF7FF70
:104DA000FB0EDBCFF8FF0800F550DF6EDF5002E1AD
:104DB00037EF2BF0250EDF5C02E02AEF2BF0030E1D
:104DC000DB6A040EDB6A050EDB6A060EDB6A070E81
:104DD000DB6A4CEC2BF02D0EDF5C0CE02B0EDF5C65
:104DE00009E0200EDF5C06E0230EDF5C03E0300EFE
:104DF000DF5C1AE1DF50300A14E0130A0FE0030A07
:104E00000AE00B0A05E0060AE4E1030EDB80E1D7C5
:104E1000030EDB82DED7030EDB84DBD7030EDB86DB
:104E2000D8D7030EDB88D5D72A0EDF5C1BE148EC10
:104E30002BF096EC2BF010E0030EDB80086809687D
:104E4000130EDBCF0DF0140EDBCF0EF0F1EC2FF0D4
:104E5000040E06C0DBFF03D0130E7FEC2BF04CECEE
:104E60002BF00BD0090EDB6AEDEC2BF003E061ECCC
:104E70002CF0FAD7090E7FEC2BF0030EDBB0DB9899
:104E80002E0EDF5C1BE14CEC2BF02A0EDF5C0BE1FD
:104E900048EC2BF096EC2BF003E1130ED1EC2BF049
:104EA0004CEC2BF00BD0090EDB6AEDEC2BF003E0A1
:104EB00061EC2CF0FAD7090ED1EC2BF0680EDF5C18
:104EC00007E14CEC2BF0680EDF5C1DE1030E18D0FF
:104ED000740EDF5C17E07A0EDF5C14E0480EDF5CD6
:104EE00006E0540EDF5C03E05A0EDF5C02E1020EC6
:104EF00007D06C0EDF5C03E06A0EDF5C04E1010E9C
:104F000024EC2CF0C9DBDF506E0A01E17FD31E0ACE
:104F100001E192D1200A01E18FD13F0A01E149D19B
:104F20001A0A01E146D10D0A01E143D1200A01E14B
:104F300040D13A0A01E13DD1200A01E13AD1260AE5
:104F400001E135D10D0A01E132D11A0A01E1D9D0CE
:104F5000200A4AE0300A1FE0460A0EE0250A01E076
:104F600083D3D950F90FE96EFF0EDA20EA6E010EF5
:104F7000EE5E000EEE5AEE5A32EC2CF0250EE66E86
:104F800095DB03E1151C01E169D32EEC2CF001E265
:104F90006BD3DB2A69D3080EDB6A040EDB500108F1
:104FA00006E2040EDB04F6EC2BF0DB508BDB080E84
:104FB000DB5009E0030EDB50010B05E172DB01E081
:104FC0004DD3080EDB6A64DBEFCFDFFFA6EC2CF0DD
:104FD00003E1151C01E142D32EEC2CF001E3DB2AA6
:104FE00060DB01E141D33AD3070EDB5002080FE149
:104FF00072EC2CF0030E39EC2CF00E0EEECFDBFF32
:105000000F0EEECFDBFF100EEECFDBFF20D0F70E42
:10501000DBCF17F0F80EDBCF18F0020E175E000E94
:10502000185AF70E17C0DBFFF80E18C0DBFF17C0C9
:10503000E9FF18C0EAFF29EC2CF0166A0E0E14C026
:10504000DBFF0F0E15C0DBFF100E16C0DBFF0E0ED0
:10505000DBCFE6FF0F0EDBCFE6FF100EDBCFE6FF68
:10506000D3EC39F0E552E552E552130E07C0DBFFF1
:10507000140E08C0DBFF060EDB5005E0130E6DECCE
:105080002CF001E26ADB91EC2CF002E2130E37DB2C
:1050900054EC2CF006E0040E6DEC2CF002E2050E50
:1050A0002EDB030EDBB005D0FCDA01E0D7D2080E10
:1050B000DB6A090EDB6A0E0EDBCFF6FF0F0EDBCFCD
:1050C000F7FF100EDBCFF8FF0800F550DF6EDF5062
:1050D00014E097EC2CF011E2A6EC2CF003E1151C87
:1050E00001E1BCD2BBDB01E3DB2A090EDB2AD9508C
:1050F0000E0FE96E000ECBDBE7D7D3DA01E1B4D2B5
:10510000ADD2C6DA110EEECFDBFF120EEDCFDBFF14
:10511000110EDBCFE6FF120EDBCFE6FFC5EC39F058
:10512000E552E552130EF3CFDBFF140EF4CFDBFF95
:10513000060EDB5004E0130ED0DB01E20EDB91EC37
:105140002CF002E2130EDBDAAFDB05E0040EC5DB68
:1051500002E2050ED4DA030EDBB005D0A2DA01E0DC
:105160007DD2080EDB6A090EDB6A110EDBCFE9FF88
:10517000120EDBCFEAFFEFCFDFFFDF5014E0D7DB0B
:1051800012E2E4DB03E1151C01E168D267DB01E315
:10519000DB2A090EDB2A110EDB2ADBCFE9FF120E18
:1051A000E8E3DB2AE6D77DDA01E15ED257D2030ECF
:1051B000DB8E070EDB0410E195DB040E5ADB0A0ED2
:1051C000EECFDBFF0B0EEECFDBFF0C0EEECFDBFFE7
:1051D0000D0EEECFDBFF6CD0070EDB5003082CE189
:1051E000030EDBAE0DD0B2DA020E76DAEFCF14F09A
:1051F000156A166A176A14AE39D01568166835D064
:10520000F70EDBCF15F0F80EDBCF16F0020E155EB1
:10521000000E165AF70E15C0DBFFF80E16C0DBFFA6
:1052200015C0E9FF16C0EAFFEFCF14F00A0E14C054
:10523000DBFF0B0EDB6A38D0070EDB50020809E1FA
:10524000030EDBAE04D059DB16AE10D00ED055DB0A
:105250000DD0030EDBAE12D079DA020E3DDAF9DAA8
:10526000166A176A15AE02D016681768E2DA0C0ED5
:1052700016C0DBFF0D0E17C0DBFF1AD0F70EDBCF19
:1052800016F0F80EDBCF17F0020E165E000E175A5E
:10529000F70E16C0DBFFF80E17C0DBFF16C0E9FFE4
:1052A00017C0EAFFD6DAC5DA0C0EDB6A0D0EDB6A30
:1052B000060EDB5005E1010EF36E050EF3CFDBFFAA
:1052C000150EDB6A160EDB6AD950370F146E000E0E
:1052D000DA20156E390E14C0DBFF3A0E15C0DBFF65
:1052E000380EDB6A080EDB6A0A0EAEDADF50780A87
:1052F00012E0200A10E0280A0CE0200A0AE03F0A27
:1053000006E00D0A02E0200A08E1020E05D0080EB0
:1053100003D0080EDF26100E97DA030EDBBE02D094
:10532000DB92DB94DB50800B24E08ADAD890030E0A
:10533000EB50000A08E6000EEE5C000EEE58000E80
:10534000EE58000EEE5815E213DA0B680C680D6883
:105350000E6873EC3AF00A0E02C0DBFF0B0E03C0BE
:10536000DBFF0C0E04C0DBFF0D0E05C0DBFF2D0EB6
:1053700008D0030EDBA202D02B0E03D0DBA408D092
:10538000200EF36E170EF3CFDBFF150EDB2A02D0D3
:10539000170EDB6A050EDB5003E1B7D901E189D0B6
:1053A0004A0E146E770E156E000E166E070EDBCFCA
:1053B00017F0186A196A1A6A17C00BF018C00CF0B7
:1053C00019C00DF01AC00EF0D3D9ABEC3AF014505E
:1053D0000224F36E15500320F46E16500420F86E6C
:1053E000F4CFF7FFF3CFF6FF0800090EF5CFDBFF90
:1053F000580EDF5C0FE1610EF36E090E7BD90AE3F4
:10540000200E146E090EDBCFE7FF1450E75E090E85
:10541000E7CFDBFF070EDBCF14F0156A166A176AB9
:105420000FDA14C00BF015C00CF016C00DF017C049
:105430000EF0EECF06F0EECF07F0EECF08F0EFCF94
:1054400009F0ABEC3AF009C0EDFF08C0EDFF07C072
:10545000EDFF06C0EFFF390EDBCFE9FFDB063A0EAA
:10546000DBCFEAFF01E2DB06090EDBCFEFFF150E13
:10547000DB2A4BD995E1030EDBA61DD06F0EDF5C56
:1054800006E1C1D918E3150EDB285BDA14D0780EDB
:10549000DF5C09E0580EDF5C06E0620EDF5C03E0D3
:1054A000420EDF5C08E1020EF36E160EF3CFDBFF57
:1054B00002D0150EDB6A030EDB50100B0EE0040E5B
:1054C000DBCF14F0050EDB50D880145406E2060E34
:1054D000DB5003E1040EDB5034DA95D90AE2050E05
:1054E000DBCFE7FF150EDB50E75E050EE7CFDBFFF6
:1054F00002D0050EDB6A040EDBCF14F0160E45D980
:10550000D880145414E2160EDBCFE6FF150EDBCF65
:10551000E6FF040EDBCFE6FF050EDB50E552E75C4D
:10552000E552D880E754E552D880E7545FD9030E9E
:10553000DB50010B0BE1080EDB5008E0B2D801E0B4
:105540008DD0080EDB50BED8080EDB6A170EDB507C
:1055500007E088D9170EF1D903E1151C01E17ED0CF
:10556000160EDB5016E07ED9300EE66E9FD802E1B3
:10557000151C74E077D9DFCFE6FFF8EC39F0E5527F
:10558000E552E552F4CF15F00001F31C02E1151CC1
:1055900065E0050EDBCF14F0160EDB50D8801454F6
:1055A00009E2050EDBCFE7FF160EDB50E75E050EC6
:1055B000E7CFDBFF300EE66E050ECBD94FE1390E9B
:1055C000DB2ADBCFE9FF3A0E01E3DB2ADBCFEAFF80
:1055D000090EEFCFDBFFDB500EE044D9090EADD949
:1055E00002E1151C3BE0390EDB2ADBCFE9FF3A0E66
:1055F000EDE3DB2AEBD755D831E1160EDBCFE6FF22
:10560000080EC3D8E552E7245DD82ED0070EDB5034
:10561000030A1CE0010A14E0030A07E07BD9DBCF90
:10562000EEFF020EDBCFEDFF1FD0F5D8196A17AEE3
:1056300002D0186819682CD8BCD819C0EEFF14D055
:10564000EAD817BE186824D8B4D80ED063D9DBCFF7
:10565000EFFF0AD07BD905E1151C03E1F368F4687C
:1056600010D0FCD801E3DB2A79D9D3EF26F0010E64
:10567000DBCF14F0020EDBCF15F014C0F3FF15C022
:10568000F4FF3B0EE15C02E2E16AE552E16ECBD051
:1056900029D9020E39EF2CF061D90800F550DF6EE0
:1056A0001200200EE66E080EA9EF2CF0F8EC39F08F
:1056B000E552E552E552F3CF14F0F4CF15F00001B6
:1056C000F31C1200146E156AD950010F4DD91450F5
:1056D000EE261550ED221200185E000E195AF70E34
:1056E00018C0DBFFF80E19C0DBFF18C0E9FF19C0B6
:1056F000EAFF1200DBCFF4FFF350F45C1200DB5042
:10570000E76E040EE7CFDBFF12000A0EDBCF14F0CA
:105710000B0EDBCF15F00C0EDBCF16F00D0EDBCF32
:1057200017F014501510161017101200130EEECFAC
:10573000DBFF140EEDCFDBFF130EDBCF14F0140EE6
:10574000DBCF15F00001800E15141200F70EDBCF31
:1057500018F0F80EDBCF19F01200050EDB50E66EE4
:10576000D950130F01D9E552E750EE6EED6A1200E1
:105770000A0EDBCF06F00B0EDBCF07F00C0EDBCFF3
:1057800008F00D0EDBCF09F01200DBCFE6FF150E9F
:10579000DBCFE6FF050EDB50E552E724E552E724B8
:1057A0001200DB50CED8010EF36E060EF3CFDBFFF6
:1057B0001200EE50EFCFEAFFE96E16C0EEFF17C001
:1057C000EEFF18C0EEFF1200D9CFE6FFDACFE6FFFA
:1057D000E1CFD9FFE2CFDAFF1200DFCFE6FFE66AC2
:1057E00053EC3BF0E552E552F3501200E76E080E21
:1057F000E7CFDBFF1200EECF14F0EECF15F0EFCFC6
:1058000016F0176A1200050EDBCF14F0150EDB50F0
:10581000D88014541200010EDBCF16F0020EDBCF3D
:1058200017F0186A1200E552E5CFDAFFE7CFD9FF8B
:1058300012000A0E14C0DBFF0B0E15C0DBFF1200B6
:10584000D9500A0FB4EF2CF0F36E070EF3CFDBFF45
:105850001200EECF14F0EFCF15F01200010EDB2A8C
:10586000020E1200FC0EDBCFE6FFFD0EDBCFE6FFE3
:105870001200145E000E155AF70E14C0DBFFF80E6E
:1058800015C0DBFF14C0E9FF15C0EAFF1200DA20E3
:10589000EA6EEF2AEECFF6FF000EEF22EECFF7FF13
:1058A000EF22EECFF8FF1200040EDBCFE6FF130E5F
:1058B000DB50E552E75C9ADFDB5004DF060EDB507D
:1058C0001200090EDB500A0DF350DF24D00FE76EF3
:1058D000090EE7CFDBFF4CEF2BF0DB50F36E050E2C
:1058E0007AEF2BF0F70EDBCF14F0F80EDBCF15F0CC
:1058F0001200DFCFE6FF56EF2BF028DF030EECDEC1
:10590000FBEF2BF0A8EC26F0E552E552E552E5520C
:1059100000091200BDDEEE50EFCFEAFFE96E010E86
:105920001200130EDB50F36E040E7AEF2BF0040E10
:10593000DB50F36E090E7AEF2BF0DBCFE6FF56EF6C
:105940002BF0E76E050EE7CFDBFF12008BDF79EF60
:105950002CF0DBCFE6FF86DF82EF2CF0D950F90F79
:10596000E96EFF0E47EF2CF0E96E000EDA20EA6ECA
:105970001200019E05D0019E09AE02D0096C018E75
:1059800009C003F0026A136A126A860E046E056A81
:1059900087EF2FF0019E08D0019E09AE05D0086C5C
:1059A000091EE86A0922018E09C003F008C002F04E
:1059B000136A126A8E0E046E056A87EF2FF0019E3D
:1059C0000CD0019E09AE09D0066C071E081E091EE8
:1059D000E86A072208220922018E09C003F008C0E4
:1059E00002F007C013F006C012F09E0E046E056AA6
:1059F00087EF2FF00F7E016AC3EC2FF0DBEC2FF066
:105A000001B66BEF2FF001A20AD001AA03D001BEAC
:105A10006BEF2FF001A477EF2FF074EF2FF001AAB6
:105A200005D001AC77EF2FF074EF2FF001A00AD072
:105A300001A808D001BE04D001A402D080EF2FF04D
:105A400084EF2FF0126A056A0F500A5C116E10E3A2
:105A500007C013F008C002F009C003F00AC010F03C
:105A60000CC007F00DC008F00EC009F0013A09D0D3
:105A70000CC013F00DC002F00EC003F00FC010F008
:105A8000116C019E01BC018E10C004F001B0B3EF97
:105A90002FF01A0E1160B3EF2FF0046A0A6A01A406
:105AA00008D0076C081E091E0A1EE86A082209228F
:105AB0000A2201AC08D0136C021E031E041EE86A01
:105AC000022203220422066A115207E00A34093234
:105AD000083207320632112EF9D707501326085024
:105AE0000222095003220A50042206C012F0019E2D
:105AF00004AE0BD0126C131E021E031E041EE86AB5
:105B00001322022203220422018E04A006D0D88090
:105B10000332023213321232102A10C004F087EF1F
:105B20002FF0016AC3EC2FF0DBEC2FF001B66BEF26
:105B30002FF001A205D001BA6BEF2FF072EF2FF01A
:105B400001BA7EEF2FF001A005D001B86BEF2FF066
:105B50007EEF2FF001B872EF2FF0056A7F0E0A2456
:105B6000046EE86A05220F50045EE86A055A1A0EB0
:105B7000106E0A6A126A136A026A036A0C50075EA0
:105B80000D50085A0E50095A000E0A5A09E70C50D7
:105B900007260D5008220E500922000E0A2201D0BD
:105BA000128AD8900736083609360A36D890123647
:105BB000133602360336102EE1D7095008100710AD
:105BC000D8A4128A87EF2FF0016AC3EC2FF0DBEC28
:105BD0002FF001B66BEF2FF001A205D001B86BEFEB
:105BE0002FF072EF2FF001AA05D001B06BEF2FF06C
:105BF00072EF2FF001B002D001A802D07EEF2FF09B
:105C0000056A0F500A24046EE86A05227E0E045EBF
:105C1000E86A055A126A136A026A036A0E50090298
:105C2000F4CF03F0F3CF02F00D500902F350132626
:105C3000F4500222000E03220E500802F3501326E5
:105C4000F4500222000E03220C500902F3501226D7
:105C5000F4501322000E022203220D500802F350CA
:105C60001226F4501322000E022203220E500702C5
:105C7000F3501226F4501322000E022203220C507D
:105C80000802F4501226000E1322022203220D50A5
:105C90000702F4501226000E13220222032287EF7D
:105CA0002FF0006A0EAE5AEF2EF00D6C0E1EE86A51
:105CB0000E22001E09AE62EF2EF0086C091EE86A83
:105CC0000922001E3DEC3BF009BE72EF2EF000AE43
:105CD000000C086C091EE86A0922046C051EE86ABB
:105CE0000522000C00BE69EF2EF00188FF0C016A4E
:105CF000C3EC2FF001B681EF2EF001A20AD001B45F
:105D000003D07F0E096E19D0800E096E16D0096A75
:105D100014D001B0FCD7870E0A60F1D77E0E0A645A
:105D2000F6D7860E0A5C04E0D89009320A2AF9D721
:105D300001A403D0096C09AEEAD71200016AC3ECD2
:105D40002FF001B6A8EF2EF001A20ED001B405D0BD
:105D50007F0E096EFF0E086E1FD0800E096E086A56
:105D60001BD0096A086A18D001B0FBD78F0E0A60F1
:105D7000EDD77E0E0A64F5D78E0E0A5C05E0D8904A
:105D8000093208320A2AF8D701A406D0086C091E85
:105D9000E86A092209AEE5D71200016AC3EC2FF0C8
:105DA00001B6D7EF2EF001A20FD001B407D07F0EBD
:105DB000096EFF0E086E076E066E25D0800E096E06
:105DC00001D0096A000EF6D701B0FBD7066A9F0E14
:105DD0000A60EBD77E0E0A64F4D79E0E0A5C07E0D9
:105DE000D89009320832073206320A2AF6D701A4BF
:105DF0000AD0066C071E081E091EE86A0722082240
:105E0000092209AEDED7120016EC2FF001B6000C05
:105E100001B0000C01B4000C010C16EC2FF001B61F
:105E2000000C01B0000C01A4000C010C016AC3ECD1
:105E30002FF0DBEC2FF001B6120001AE08D001A06C
:105E400004D001A802D001801200019012000F506E
:105E50000A5C0BE10E50095C08E10D50085C05E19D
:105E60000C50075C02E101801200D8A002D0018E24
:105E700010D00A500FC00AF00F6E09500EC009F082
:105E80000E6E08500DC008F00D6E07500CC007F0E4
:105E90000C6E0F500A5C10E0FF0F09E0019001B496
:105EA00003D001AE0184120001AE019412000F2A4A
:105EB000D8900E320D320C320C50075E0D50085A3D
:105EC0000E50095A09BEEAD7D89007360836093667
:105ED0000A2EF8D7C8D77F0E0A6EFF0E096E086E1D
:105EE000076E12007F0E01BEFF0E0A6E02D07F0EFB
:105EF0000A6E800E096E086A076AF3D701AE04D0F5
:105F0000800E0A6E096AF7D70A6A096AF4D7035045
:105F1000021013101210F8E005BEF0D703BE0CD02B
:105F200004500510EBE0D8901236133602360336D3
:105F30000406D8A00506F2D70550D4E10428D2E023
:105F400012AE11D07F0E121402E113A00CD0132A4E
:105F5000E86A0222032207E3D880033202321332B6
:105F6000042A0428BFE00450C9E013C007F002C0AF
:105F700008F00334096E04300A6E09320A9E01BE2D
:105F80000A8E71EF2FF009360A3602E30184017E92
:105F900006E101800A6A096A086A076A12000A288B
:105FA00003E0D88009321200D890093202E1018260
:105FB0001200018612000E360F3602E3018C017EBC
:105FC00006E101880F6A0E6A0D6A0C6A12000F283A
:105FD00003E0D8800E321200D8900E32EAE1018A36
:105FE000120009C013F008C012F008500D02F4CFDF
:105FF00007F0F3CF06F009500E02F4CF09F0F3CF0B
:1060000008F00D02F3500726F4500822E86A09222E
:1060100012500E02F3500726F4500822E86A0922B3
:106020000EAE17EF30F01250085E1350095A13AE3F
:10603000000C0D50085E0E50095A000C0080808044
:106040008080800000C0C0C0C0C0C00000E0E0E0B0
:10605000E0E0E00000F0F0F0F0F0F00000F8F8F818
:10606000F8F8F80000FCFCFCFCFCFC0000FEFEFE66
:10607000FEFEFE0000FFFFFFFFFFFF000010181CE8
:106080001E1C1810000103070F070301040E1F0E4A
:106090000E0E0E0E0E0E0E0E0E1F0E0402040E112C
:1060A0001F100E0008040E111F100E0008040E0130
:1060B0000F110F0002050200000000008082858899
:1060C0008B8E9194979A9DA0A2A5A8ABADB0B3B5C5
:1060D000B8BBBDC0C2C5C7C9CCCED0D2D4D6D8DA21
:1060E000DCDEE0E2E3E5E6E8E9EBECEDEEEFF0F133
:1060F000F2F3F4F5F5F6F6F7F7F7F7F7F8F7F7F741
:10610000F7F7F6F6F5F5F4F3F2F1F0EFEEEDECEB70
:10611000E9E8E6E5E3E2E0DEDCDAD8D6D4D2D0CEB8
:10612000CCC9C7C5C2C0BDBBB8B5B3B0ADABA8A5DF
:10613000A2A09D9A9794918E8B888582807D7A7794
:1061400074716E6B6865625F5D5A5754524F4C4A6A
:106150004744423F3D3A383633312F2D2B292725EE
:1061600023211F1D1C1A19171614131211100F0EBC
:106170000D0C0B0A0A09090808080808080808088D
:10618000080809090A0A0B0C0D0E0F10111213143E
:106190001617191A1C1D1F21232527292B2D2F31D6
:1061A0003336383A3D3F4244474A4C4F5254575A8F
:1061B0005D5F6265686B6E7174777A7D00010203C2
:1061C0000405060708090A0B0C0D0E0F1011121317
:1061D0001415161718191A1B1C1D1E1F2021222307
:1061E0002425262728292A2B2C2D2E2F30313233F7
:1061F0003435363738393A3B3C3D3E3F40414243E7
:106200004445464748494A4B4C4D4E4F50515253D6
:106210005455565758595A5B5C5D5E5F60616263C6
:106220006465666768696A6B6C6D6E6F70717273B6
:106230007475767778797A7B7C7D7E7F80818283A6
:106240008485868788898A8B8C8D8E8F9091929396
:106250009495969798999A9B9C9D9E9FA0A1A2A386
:10626000A4A5A6A7A8A9AAABACADAEAFB0B1B2B376
:10627000B4B5B6B7B8B9BABBBCBDBEBFC0C1C2C366
:10628000C4C5C6C7C8C9CACBCCCDCECFD0D1D2D356
:10629000D4D5D6D7D8D9DADBDCDDDEDFE0E1E2E346
:1062A000E4E5E6E7E8E9EAEBECEDEEEFF0F1F2F336
:1062B000F4F5F6F7F8F9FAFBFCFDFEFFFFFFFFFF30
:1062C000FFFFFFFFFFFFFFFFFFFFFFFFFFFFFFFFDE
:1062D000FFFFFFFFFFFFFFFFFFFFFFFFFFFFFFFFCE
:1062E000FFFFFFFFFFFFFFFFFFFFFFFFFFFFFFFFBE
:1062F000FFFFFFFFFFFFFFFFFFFFFFFFFFFFFFFFAE
:10630000FFFFFFFFFFFFFFFFFFFFFFFFFFFFFFFF9D
:10631000FFFFFFFFFFFFFFFFFFFFFFFFFFFFFFFF8D
:10632000FFFFFFFFFFFFFFFFFFFFFFFFFFFFFFFF7D
:10633000FFFFFFFFFFFFFFFFFFFFFFFF0000000069
:10634000000000000000000000000000000000004D
:10635000000000000000000000000000000000003D
:10636000000000000000000000000000000000002D
:10637000000000000000000000000000000000001D
:10638000000000000000000000000000000000000D
:1063900000000000000000000000000000000000FD
:1063A00000000000000000000000000000000000ED
:1063B00000000000000000000000000008090B0DB4
:1063C0000F11131517181A1C1E2022242627292BFB
:1063D0002D2F31333536383A3C3E4042444547490B
:1063E0004B4D4F51535456585A5C5E60626365671B
:1063F000696B6D6F71727476787A7C7E808183852B
:1064000087898B8D8F90929496989A9C9E9FA1A33A
:10641000A5A7A9ABADAEB0B2B4B6B8BABCBDBFC14A
:10642000C3C5C7C9CBCCCED0D2D4D6D8DADBDDDF5A
:10643000E1E3E5E7E9EAECEEF0F2F4F6F8F6F4F27F
:10644000F0EEECEAE9E7E5E3E1DFDDDBDAD8D6D42C
:10645000D2D0CECCCBC9C7C5C3C1BFBDBCBAB8B6FC
:10646000B4B2B0AEADABA9A7A5A3A19F9E9C9A98CC
:10647000969492908F8D8B8987858381807E7C7A9C
:1064800078767472716F6D6B6967656362605E5C6C
:106490005A58565453514F4D4B4947454442403E3C
:1064A0003C3A38363533312F2D2B2927262422200C
:1064B0001E1C1A18171513110F0D0B094CD8B43CDC
:1064C000204672616D652045727265757220657433
:1064D000204F766572666C6F7720646574656374AF
:1064E000696F6E203A200020506F727420636F6DC8
:1064F0006D203139323030626473206F7576657289
:106500007400204465706861736167652053696732
:106510006E616C20414439383530203A20002045E6
:10652000534320706F757220736F727469720D001F
:10653000204361707475726520546175782073759D
:10654000722041444330200020496E697420436F1B
:106550006D70617261746F727320312065742032C6
:10656000203A2000204661637465757220444453CC
:1065700020414439383530203D2000205573616773
:106580006520513D31304D687A20783428504C4C8C
:10659000290D002045727265757220536169736917
:1065A000652E2E2E2E2E0D0020496E697420436F0D
:1065B0006E734672657120314B687A09002046611E
:1065C00063746575722044445320504943203D2034
:1065D0000020496E7465726661636520766961208A
:1065E0005465726D696E616C2052533233322045AE
:1065F000542F4F5520766961204A6F79737469630F
:106600006B202B204C43440D002047616D6D6520AD
:106610006465203120612032352E303030487A20B8
:10662000200D00202031384634364B32325F44444E
:10663000535F3133303531395F41444335625F4117
:1066400044393835305F4C43445F52533233325F04
:106650004A6F79737469636B5F4331382E630D0041
:10666000FF0EE3CFEAFFE552FF0EE3CFE9FFE5526D
:10667000E66AE66AD9CFE6FFDACFE6FFFC0EE12450
:10668000D96EFF0EE220DA6EE66AE66AE66A200E4E
:10669000EF5C06E0090EEF5C03E0EF6603D03FD04D
:1066A000EE50F5D72D0EEF5C03E1FF0EE32A03D089
:1066B0002B0EEF5C01E1EE502F0EEF6424D03A0E6A
:1066C000EF6021D0D890F90EE336FA0EE336FD0ED6
:1066D000DECFE3FFFE0EDDCFE3FFD890F90EE33609
:1066E000FA0EE336D890F90EE336FA0EE336FD0ED5
:1066F000E350DE26FE0EE350DD22300EEE5CDE2699
:10670000000EDD22D9D7FF0EE3CFE8FFE85207E005
:10671000F90EE31EE32AFA0ED8B4E306E31EE552AF
:10672000E552E552FF0EE3CFDAFFE552FF0EE3CF6D
:10673000D9FFE552E1CFE9FFE2CFEAFFED52ED529A
:10674000EECFF3FFEFCFF4FF1200FF0EE3CFEAFF2F
:10675000E552FF0EE3CFE9FFE552E66AE66AE66A34
:10676000E66AD9CFE6FFDACFE6FFFA0EE124D96E6A
:10677000FF0EE220DA6EE66AE66AE66AE66AE66A32
:10678000200EEF5C06E0090EEF5C03E0EF6603D03D
:106790006BD0EE50F5D72D0EEF5C03E1FF0EE32A30
:1067A00003D02B0EEF5C01E1EE502F0EEF6444D0CE
:1067B0003A0EEF6041D0D890F50EE336F60EE33690
:1067C000F70EE336F80EE336FB0EDECFE3FFFC0EEA
:1067D000DECFE3FFFD0EDECFE3FFFE0EDDCFE3FFF6
:1067E000DD52DD52D890F50EE336F60EE336F70EA5
:1067F000E336F80EE336D890F50EE336F60EE336C0
:10680000F70EE336F80EE336FB0EE350DE26FC0E01
:10681000E350DE22FD0EE350DE22FE0EE350DD22C9
:10682000DD52DD52300EEE5CDE26000EDE22DE2270
:10683000DD22DD52DD52B9D7FF0EE3CFE8FFE8528B
:1068400013E0F50EE31EF60EE31EF70EE31EF80E40
:10685000E31EF50EE32A08E1F60EE32A05E1F70E42
:10686000E32A02E1F80EE32AE552E552E552E55249
:10687000E552D9CFE9FFDACFEAFFEECF06F0EECF4F
:1068800007F0EECF08F0EFCF09F0FF0EE3CFDAFF0D
:10689000E552FF0EE3CFD9FFE552E552E552120073
:1068A000D9CFE6FFDACFE6FFFA0EE3CFD9FFFB0E32
:1068B000E3CFDAFFFD0EE35209E72D0EDE6EFC0E8C
:1068C000E31EE32AFD0ED8B4E306E31EE652E652C9
:1068D000E652FD0EE124E76EFF0EE220E46EE65282
:1068E000F70EE3CFE6FFF70EE3CFE6FFC0EC34F0A0
:1068F000F90EE124E96EFF0EE220EA6EB0EC34F00E
:106900000AE1ADEC34F009E1B0EC34F008E1ADECB3
:1069100034F007E108D0BBEC34F0B6EC34F0BBEC5B
:1069200034F0B6EC34F0BBEC34F0DE6AF90EE1265C
:10693000FF0EE222FF0EE3CFDAFFE552FF0EE3CFB8
:10694000D9FFE552FC0EE124E96EFF0EE220EA6E6B
:10695000EECFF3FFEFCFF4FF1200EF380F0B120072
:10696000EF500F0B02E1EE52D8841200EF380F0BFC
:10697000300FDE6E1200EE500F0B300FDE6E120085
:10698000FC0EE3CFE9FFFD0EE3CFEAFF100EE66E4B
:10699000EE6AEE6AEF6AD890FD0EE336FE0EE3363D
:1069A000ED36ED36EF36FF0EE30609E0E1EC34F0AC
:1069B000EE52E1EC34F0EE52E1EC34F0EDD7E56E5E
:1069C0001200030EEF24E8B6EF6E300EEF24E8BE9F
:1069D000EF6E000CD9CFE6FFDACFE6FFF80EE3CF7B
:1069E000D9FFF90EE3CFDAFFE652E652E652E6525D
:1069F000E652FB0EE124E76EFF0EE220E46EE65263
:106A0000F30EE3CFE6FFF30EE3CFE6FFF30EE3CFA3
:106A1000E6FFF30EE3CFE6FF6FEC35F0F50EE12471
:106A2000E96EFF0EE220EA6E5CEC35F019E15FECF6
:106A300035F018E15CEC35F017E15FEC35F016E16C
:106A40005CEC35F015E15FEC35F014E15CEC35F011
:106A500013E15FEC35F012E15CEC35F011E112D09E
:106A600065EC35F06AEC35F065EC35F06AEC35F044
:106A700065EC35F06AEC35F065EC35F06AEC35F034
:106A800065EC35F06AEC35F0DE6AF50EE126FF0EB6
:106A9000E222FF0EE3CFDAFFE552FF0EE3CFD9FF8C
:106AA000E552FA0EE124E96EFF0EE220EA6EEECF27
:106AB000F3FFEFCFF4FF1200EF380F0B1200EF508F
:106AC0000F0B02E1EE52D8841200EF380F0B300F9B
:106AD000DE6E1200EE500F0B300FDE6E1200FA0E5B
:106AE000E3CFE9FFFB0EE3CFEAFF200EE66EEE6A8E
:106AF000EE6AEE6AEE6AEF6AD890FB0EE336FC0EA1
:106B0000E336FD0EE336FE0EE336ED36ED36ED36BA
:106B1000ED36EF36FF0EE3060FE09EEC35F0EE5259
:106B20009EEC35F0EE529EEC35F0EE529EEC35F0D8
:106B3000EE529EEC35F0E1D7E56E1200030EEF2425
:106B4000E8B6EF6E300EEF24E8BEEF6E000CD9CF42
:106B5000E6FFDACFE6FFE1CFD9FFE2CFDAFF130E8F
:106B6000E12402E3E168E652E16E0C0EDB6AD950E3
:106B7000FA0FE96EFF0EDA20EA6E080EEECFDBFFA9
:106B8000090EEECFDBFF0A0EEECFDBFF0B0EEECFD2
:106B9000DBFF1FD9D950080F17D9EECFE6FFEECF94
:106BA000E6FFEECFE6FFEFCFE6FFF0EC36F0146E37
:106BB000060EE15C02E2E16AE552E16E1450DF6E1E
:106BC000020EDF5C01E0BCD0050EDBCF16F0060E36
:106BD000DBCF17F0F80EDB50165C146EF90EDB50AD
:106BE0001758156E7F0E145E000E155A0D0E14C048
:106BF000DBFF0E0E15C0DBFF0D0E0E0EDBCF15F00A
:106C00000001800E15140AE0010EF36E0C0EF3CF96
:106C1000DBFF070EDB5001E098D09DD00D0EDBCFDF
:106C200014F00E0EDBCF15F0D890155004E6170EB9
:106C3000145C000E155801E39ED0186819687F0E89
:106C40001A6E1B6A0D0EDB501F0B18C014F019C012
:106C500015F01AC016F01BC017F007E0D8901732D5
:106C6000163215321432E806F9E10F0E14C0DBFFBC
:106C7000100E15C0DBFF110E16C0DBFF120E17C081
:106C8000DBFF0F0EDBCF14F0100EDBCF15F0110E73
:106C9000DBCF16F0120EDBCF17F0D950010F94D8CE
:106CA000EE501416EE501516EE501616EE5017163E
:106CB000145015101610171002E1000E01D0010E2D
:106CC000E76E0C0EE7CFDBFFDB5055E0186A196A60
:106CD000800E1A6E1B6A010E1C6E1D6A1E6A1F6AE8
:106CE000D9500F0F71D8EE501C26EE501D22EE50D9
:106CF0001E22EE501F221C50185C146E1D50195895
:106D0000156E1E501A58166E1F501B58176ED9500C
:106D1000010F5AD81450EE161550EE161650EE16F6
:106D20001750EE16D950080FE66E000EDA20E66E08
:106D300050D87EEC37F0E552E552E552E5521BD0D3
:106D4000DF0419E1070EDB5006E0146A156A166AC3
:106D5000800E176E04D0146A156A166A176A080E38
:106D600014C0DBFF090E15C0DBFF0A0E16C0DBFFE7
:106D70000B0E17C0DBFFF60EDBCFE9FFF70EDBCF04
:106D8000EAFF0C0EDBCFEFFF080EDBCF14F0090E8D
:106D9000DBCF15F00A0EDBCF16F00B0EDBCF17F0B2
:106DA00014C006F015C007F016C008F017C009F0AF
:106DB000130EE15C02E2E16AE552E16EE552E5CFD5
:106DC000DAFFE7CFD9FF1200E96E000EDA20EA6E93
:106DD0001200D950010FE66E000EDA20E66E1200A6
:106DE000D9CFE6FFDACFE6FFE1CFD9FFE2CFDAFF76
:106DF000E652146815687F0E166E176AD950FA0F9E
:106E0000E96EFF0EDA20EA6EEE501416EE501516FB
:106E1000EE501616EE5017166AD814C0EEFF15C0C5
:106E2000EEFF16C0EEFF17C0EEFFFD0EDB50800B2D
:106E300002E0010E01D0000EE66E59D8060EE926DA
:106E4000000EEA22E552E750EF6EFC0EDBCF14F0A5
:106E5000FD0EDBCF15F0D89014361536FC0E14C09D
:106E6000DBFFFD0E15C0DBFFDB50E66E40D8040EE5
:106E7000E926000EEA22E552E750EE6EED6AFD0EBD
:106E8000DB50146E156AFF0E141818E1155016E148
:106E90002ED8EECF14F0EECF15F0EECF16F0EFCFE8
:106EA00017F0145015101610171006E0210E0001EF
:106EB000EA6FEB6B800E0BD0040E09D0FD0EDB5099
:106EC00008E115D8EE6AEE6AEE6AEE6A010EDF6E30
:106ED00006D0020EDF6E0BD8EE52EE52EE8EDF5071
:106EE000E552E552E5CFDAFFE7CFD9FF1200F80E01
:106EF000DBCFE9FFF90EDBCFEAFF1200D9CFE6FFC7
:106F0000DACFE6FFE1CFD9FFE2CFDAFF5BD8153465
:106F100011E21450FE08000E15540CE276D805E07C
:106F20006CD8800EEE6EEE6847D067D8800EEE6E9D
:106F30007F0E0ED047D8D890155004E6010E145C91
:106F4000000E15580BE261D805E057D8EE6A800EA6
:106F5000EE6E32D052D8EE6AEE6A2ED047D8EECF1F
:106F600014F0EECF15F0EECF16F0EFCF17F032D8C9
:106F700014C0EEFF15C0EEFF16C0EEFF17C0EEFF07
:106F800021D81450010B05E025D8020E3AD8EF8E17
:106F900004D020D8020E35D8EF9E14D8D8901532E0
:106FA000143218D8030E2DD814C0EFFF1AD804E0FD
:106FB00011D8030E26D8EF8EE552E5CFDAFFE7CFE2
:106FC000D9FF120013D8040E1CD8EECF14F0EFCF67
:106FD00015F01200FA0EDBCFE9FFFB0EDBCFEAFF64
:106FE000120004D8060E0DD8EF501200FC0EDBCFB5
:106FF000E9FFFD0EDBCFEAFF1200ECDFEE6AEE6A7E
:107000001200E926000EEA221200220E0001EA6FA9
:10701000EB6BF1EF37F0D9CFE6FFDACFE6FFE1CF48
:10702000D9FFE2CFDAFF060EE12402E3E168E6527F
:10703000E16ED950050FE66E000EDA20E66E000E06
:10704000E66EE66AD950FA0FE96EFF0EDA20EA6EB4
:10705000EECFE6FFEECFE6FFEECFE6FFEFCFE6FFA7
:10706000A7EC35F0146E080EE15C02E2E16AE5522D
:10707000E16E1450010E06C0DBFF020E07C0DBFFFD
:10708000030E08C0DBFF040E09C0DBFF050EDB505A
:107090002AE0040EDB50800B26E1146A156A800E8C
:1070A000166E3F0E176ED950010FE96E000EDA20F2
:1070B000EA6EEECF07F0EECF08F0EECF09F0EFCF9B
:1070C0000AF014C00CF015C00DF016C00EF017C079
:1070D0000FF0FBEC2CF00AC0EDFF09C0EDFF08C07B
:1070E000EDFF07C0EFFF010EDBCF14F0020EDBCF88
:1070F00015F0030EDBCF16F0040EDBCF17F014C033
:1071000006F015C007F016C008F017C009F0060E0B
:10711000E15C02E2E16AE552E16EE552E5CFDAFFB9
:10712000E7CFD9FF120020204164393835305F4362
:107130006F6E74726F6C203D2025303258206F7551
:10714000747075742053494E555320414439383575
:107150003020257320B0200D00205265676C6167D8
:107160006520636F6E7369676E65204144393835F9
:10717000302061202530386C642020736F697420C2
:1071800025732020487A0D00205265676C61676581
:1071900020636F6E7369676E6520414439383530FE
:1071A0002061202530386C6420706172206465662F
:1071B0006175742020736F69742025732020487ACC
:1071C0000D00257320566572746963616C203D253E
:1071D0003034642020486F72697A6F6E74616C3D40
:1071E00025303464200D2076616C657572207365DE
:1071F00075696C206261733D202530346420736FA3
:107200006974200031384634364B323220444453BE
:10721000204331380020342E3039365600FF0E0E10
:10722000F66E000EF76E000EF86E00010900F550C4
:10723000E56F0900F550E66F03E1E56701D03DD049
:107240000900F550E06F0900F550E16F0900F550B5
:10725000E26F09000900F550E96E0900F550EA6E89
:10726000090009000900F550E36F0900F550E46FCB
:1072700009000900F6CFE7F0F7CFE8F0F8CFE9F022
:10728000E0C0F6FFE1C0F7FFE2C0F8FF0001E35302
:1072900002E1E45307E00900F550EE6EE307F8E27F
:1072A000E407F9D7E7C0F6FFE8C0F7FFE9C0F8FF49
:1072B0000001E507000EE65BBFD71200D9CFE6FF5D
:1072C000DACFE6FFE1CFD9FFE2CFDAFFE652E652AE
:1072D000E652E652D950F90F146EFF0EDA20156E01
:1072E00014C0DEFFDD6EDECFE6FFDDCFE6FFF90E78
:1072F000DBCFE6FFFA0EDBCFE6FFFB0EDBCFE6FFD0
:10730000FC0EDBCFE6FFFD0EDBCFE6FFBEEC26F08A
:10731000146E070EE15C02E2E16AE552E16E145080
:10732000020EF3CFDBFF030EF4CFDBFF020EDBCF49
:1073300014F0030EDBCF15F014C0F3FF15C0F4FFFB
:10734000040EE15C02E2E16AE552E16EE552E5CF4E
:10735000DAFFE7CFD9FF1200FB0EE3CFF6FFFC0EFA
:10736000E3CFF7FFFD0EE3CFF8FFFE0EE3CFE9FF1B
:10737000FF0EE3CFEAFFE9CFF3FFEACFF4FF090006
:10738000F5CFEFFFEE66FBD71200FE0EE3CFE9FF6D
:10739000FF0EE3CFEAFFF36AF46AEE5203E0F34A2A
:1073A000F42AFBD71200FF0EE3CFF8FFE552FF0EE1
:1073B000E3CFF7FFE552FF0EE3CFF6FFE552E66AB3
:1073C000E66AE66A0900F55209E0FD0EE32A05E1E6
:1073D000FE0EE32A02E1FF0EE32AF4D7FD0EE3CF0F
:1073E00007F0FE0EE3CF08F0FF0EE3CF09F0120026
:1073F000D9CFE6FFDACFE6FFE1CFD9FFE2CFDAFF60
:10740000FB0EDBCF14F0FC0EDBCF15F00001800E7D
:1074100015141AE1FB0EDBCFE9FFFC0EDBCFEAFF10
:10742000EECFF3FFEDCFF4FFEE2A000EEF22F3CF05
:10743000E9FFF4CFEAFFFD0EDBCFEFFFEF50156A57
:10744000F36E15C0F4FF10D0FB0EDB50FE0806E112
:10745000FD0EDBCFE6FF83EC3BF005D0FD0EDBCF6E
:10746000E6FF03EC00F0E552E552E5CFDAFFE7CFA7
:10747000D9FF1200D9CFE6FFDACFE6FFE1CFD9FF7F
:10748000E2CFDAFFAC6AAB6AFD0EDBB0AC88DBA200
:1074900002D0AC8CAB8CDBB4AC8EDBA602D0AB885C
:1074A00001D0AB8ADBB8AC84DBBAAB86DBAC02D0F4
:1074B0009D8A01D09D9ADBAE02D09D8801D09D9817
:1074C000FB0EDB50AF6EFC0EDBCF15F015C014F0D9
:1074D000156A1450B06EAC8AAB8EE552E5CFDAFF78
:1074E000E7CFD9FF120006500B02F3CF02F0F4CF22
:1074F00003F00C02F3500326000EF420046E065035
:107500000D02F3500426000EF420056E06500E0204
:10751000F350052607500B02F3500326F4500422C3
:10752000000E052207500C02F3500426F4500522E9
:1075300007500D02F350052608500B02F3500426A5
:10754000F450052208500C02F350052609500B0296
:10755000F35005261200056A046A036A026A200EC7
:10756000E76ED890063607360836093602360336F7
:10757000043605360B50025C0C5003580D5004586D
:107580000E50055809E30B50025E0C50035A0D5083
:10759000045A0E50055A062AE72EE4D71200D9CF16
:1075A000E6FFDACFE6FFE1CFD9FFE2CFDAFFE6521E
:1075B000F20E0001EC17ABAC03D0EC91ABB0EC8158
:1075C000ABB4EC85ABB2EC87AE50DF6EDF50E5526A
:1075D000E552E5CFDAFFE7CFD9FF1200D9CFE6FFBA
:1075E000DACFE6FFE1CFD9FFE2CFDAFFE652E6528B
:1075F000FC0EDBCFDEFFDBCFDDFF010EDB50CF6EFD
:10760000DF50CE6EE552E552E552E5CFDAFFE7CF27
:10761000D9FF1200D9CFE6FFDACFE6FFE1CFD9FFDD
:10762000E2CFDAFFE652E652FC0EDBCFDEFFDBCF25
:10763000DDFF010EDB50D76EDF50D66EE552E5520E
:10764000E552E5CFDAFFE7CFD9FF1200D9CFE6FF49
:10765000DACFE6FFE1CFD9FFE2CFDAFFACAC04D05E
:10766000AC900001ECB3AC80FD0EDB50AD6EE5528A
:10767000E5CFDAFFE7CFD9FF1200056A046A100EE2
:10768000E76ED89008360936043605360D50045C8E
:107690000E50055805E30D50045E0E50055A082A99
:1076A000E72EF0D71200F36AF46AFF0EE124E96EC8
:1076B000FF0EE220EA6EED6607D02F0EEF6404D0D5
:1076C0003A0EEF6001D0F32A1200380EF36E00EE8E
:1076D00000F00F0E01D81200EA6002D0EE6AFCD76B
:1076E000F350E9601200EE6AFCD71EEE00F02EEEB9
:1076F00000F0F86A019C0FEC39F0B5EC3BF081EC3E
:107700001DF0FBD71200FF0EE350ACBA04D0AF6AF5
:10771000AB8EAC8A949CACA2FED7AD6EF36EF46ACD
:107720001200FF0EE350E84E1200000000D000D01F
:1077300000D0E82EFAD71200C450176E166AC35054
:107740001610F36E17C0F4FF1200303132333435A7
:107750003637383961626364656600FFC250020BD8
:1077600001E0010E1200C28212001200C064E76440
:1077700002651E653065486564657B659365A8652F
:10778000BD65D165096623660100020005000A0097
:10779000140032006400C800F401EE02E803E204C1
:1077A000DC05D606D007C409BE0AB80BAC0DA00F85
:1077B000941188137C1570176419581B4C1D401FB9
:1077C000342128231C251027F82AE02EC832B03691
:1077D000983A803E68425046384A204E0852F0554A
:1077E000D859C05DA86190657869606D4871307541
:1077F0001879007DE880D084B888A08C8890709437
:107800005898409C04A6C8AF0000010002000A007E
:10781000190032006400FA00F401EE02E8030000EF
:107820000100020005000A0032006400FA00F401C1
:10783000E8038813000000000100000005000000BC
:107840000A0000003200000064000000F4010000A3
:10785000E80300008813000010270000A086010044
:10786000BC6050726F6A657420433138203A203111
:10787000384634364B32325F4444535F41443938E2
:1078800035305F6A6F79737469636B2E6D63700D49
:1078900000000000000000000000000000000000E8
:1078A00000000000000000000000000000000000D8
:1078B0000000D90831323334353637383930313277
:1078C000333435000000000000000000000000001C
:1078D00000FFFFFFFFFFFFFFFFFFFFFFFFFFFFFFB7
:1078E000FFFFFFFFFFFFFFFFFFFFFFFFFFFFFFFFA8
:1078F000FFFFFFFFFFFFFFFFFFFFFFFFFFFFFFFF98
:10790000FFFFFFFFFFFFFFFFFFFFFFFFFFFFFFFF87
:10791000FFFFFFFFFFFFFFFFFFFFFFFFFFFFFFFF77
:0200000400F00A
:100000002031384634364B32322034304D687A2035
:10001000513D31304D687A20504C4C78340D000001
:100020002053696E7573202020202020202020205E
:10003000202020202020202020202020200D000013
:100040002043617272652020202020202020202063
:10005000202020202020202020202020200D0000F3
:1000600020547269616E676C65202020202020205A
:10007000202020202020202020202020200D0000D3
:100080002044656E742064652073636965202020B8
:10009000202020202020202020202020200D0000B3
:1000A00020526576657273652064656E74206465A0
:1000B000207363696520202020202020200D00006F
:1000C0002052656374616E676C65206628546175A3
:1000D000782920202020202020202020200D000012
:1000E000205265676C6167652054617578205265A0
:1000F0006374616E676C6520656E2025200D0000BD
:10010000205265676C6167652046726571204444C2
:1001100053204144393835302061203A20200000F6
:100120002043686F697820467265712E50494344B8
:1001300044532031207061726D692036330D000008
:10014000205265676C6167652046696E204672655E
:100150007175656E6365205049434444530D00003A
:10016000205265676C616765204672657120444462
:1001700053204144393835302061203A2020000096
:1001800020496E697420736F72746965204441431D
:100190003D20536575696C20486175743A200000F4
:1001A000204D504C4142204944452056382E39308C
:1001B0002C4331382056332E34342E20200D0000AD
:1001C0002056657273696F6E2031392F30352F31AB
:1001D0003320207061756C666A756A6F200D0000AF
:1001E00020446570686173616765205369676E615B
:1001F0006C2041443938353020202020200D00006B
:1002000030202D2D2D2D2D2D2D2D2D2D2D2D2D2D28
:10021000202020202053494E5553202020202020EC
:100220002020202020436172726520202020202081
:100230002020202020547269616E676C6520202088
:100240002044656E74732064652053434945202023
:100250007265762044656E74206465205343494579
:100260002020202052656374616E676C6520202019
:100270004D6F646520444453204144393833352060
:100280005265676C2E544155582052656374616EF7
:1002900043686F6978204672657120466978657396
:1002A0005265676C2E467265712050494344445331
:1002B0005265676C2E46726571204144393835307D
:1002C0004630206F75204631202041443938353082
:1002D0003133202D2D2D2D2D2D2D2D2D2D2D2D2D51
:1002E00056657273696F6E2031392F30352F313377
:1002F0004465706861736167652041443938353001
:10030000FFFFFFFFFFFFFFFFFFFFFFFFFFFFFFFFFD
:10031000FFFFFFFFFFFFFFFFFFFFFFFFFFFFFFFFED
:10032000FFFFFFFFFFFFFFFFFFFFFFFFFFFFFFFFDD
:10033000FFFFFFFFFFFFFFFFFFFFFFFFFFFFFFFFCD
:10034000FFFFFFFFFFFFFFFFFFFFFFFFFFFFFFFFBD
:10035000FFFFFFFFFFFFFFFFFFFFFFFFFFFFFFFFAD
:10036000FFFFFFFFFFFFFFFFFFFFFFFFFFFFFFFF9D
:10037000FFFFFFFFFFFFFFFFFFFFFFFFFFFFFFFF8D
:10038000FFFFFFFFFFFFFFFFFFFFFFFFFFFFFFFF7D
:10039000FFFFFFFFFFFFFFFFFFFFFFFFFFFFFFFF6D
:1003A000FFFFFFFFFFFFFFFFFFFFFFFFFFFFFFFF5D
:1003B000FFFFFFFFFFFFFFFFFFFFFFFFFFFFFFFF4D
:1003C000FFFFFFFFFFFFFFFFFFFFFFFFFFFFFFFF3D
:1003D000FFFFFFFFFFFFFFFFFFFFFFFFFFFFFFFF2D
:1003E000FFFFFFFFFFFFFFFFFFFFFFFFFFFFFFFF1D
:1003F000FFFFFFFFFFFFFFFFFFFFFFFFFFFFFFFF0D
:020000040030CA
:0E0000000033193C009D84000FC00FE00F403C
:020000040020DA
:08000000FFFFFFFFFFFFFFFF00
:00000001FF
